:020000041100E9
:103000007FB50023284C294D03932800217C284AB2
:1030100001F0D5FA002812D103232800217C03AA4D
:1030200001F074FA00280AD1224B039A9A4206D181
:10303000214B2248E360224B636104B070BD02263D
:10304000217CFE2228001F4B009601F031FA002857
:1030500001D00020F1E71C4BA2899A42F9D1217CD2
:10306000FF222800194B009601F022FA0028F0D127
:10307000E389174A934203D1164B17486361DCE793
:10308000164A9342E5D1164B164A1B68934206D95D
:10309000C02304222800217C9B0001F072FA124B0D
:1030A00012486361C9E7C046A061FF1FD441FF1FFA
:1030B00081370000595953005959832090BE00119F
:1030C000F1410011AC61FF1F59590000AE61FF1FB3
:1030D00083050000A541001170BE0011821500009B
:1030E000C461FF1F87130000AD42001180BE0011B4
:1030F000002370B51A4E1B4C30006361637401F0FD
:1031000085F9402323744B2B0CD9CC233821AC22D6
:1031100030009B01217401F034FA00280AD0002508
:1031200025740CE0FFF76CFF051E08D1237C0433E7
:10313000DBB2E7E70C4B0D4D63610D4BE381236878
:10314000002B08D1002D06D00C222900200008F009
:10315000ABFC2B7B6374300001F096F970BDC04668
:10316000D441FF1FA061FF1F4542001160BE001146
:10317000AAAAFFFFF7B5164B0192C318021D002043
:10318000009388235B05D3181B685C1C1AD09CB283
:10319000402C18D88D781E0CAC466746CD782D0291
:1031A0003D43AE4206D1019800280ED110000C70AC
:1031B000240A4C7003249BB20733A343D218009B0C
:1031C0009A42DED3FEBD4432F9E71000FAE7C0466A
:1031D000FC0F0000802213B503000324019189B283
:1031E000520107319B18A14304305A1A88235B050A
:1031F000C3181B68591C03D190429241104016BD60
:1032000099B2402907D80B000733A343C018904256
:10321000ECD30020F3E74430F9E7134B134A1B6863
:10322000126810B5FA24934201D81A00F824104B02
:10323000E4021B689A4210D813000E4A12689A42A0
:103240000ED3013307D1F823DB029C4203D10A4994
:10325000054808F089FC200010BDFC24E402ECE7DE
:10326000FE24E402F7E7C04600C0071100D00711B2
:1032700000E0071100F00711FFFFFF7FF0B59BB0E2
:10328000150004900391402A00D9A0E006AB5980B4
:103290001A80FFF7C2FF0400042816D9002206A9ED
:1032A000FFF768FF052810D906AB1B88AB420CD18D
:1032B000002D07D0514B2A000499C01808F0B4FA29
:1032C000002802D101201BB0F0BD06AB1D802000FC
:1032D0000699FFF77FFF041E7BD1069B0793FFF73C
:1032E0009CFF80235B01C618802307001B039E42BE
:1032F00001D3F826F60288235B05F31801931B68B7
:10330000013302D0019808F03FFB3D49019808F0D5
:103310002BFC3B1D0293331D05938822029B520513
:103320009B181B6808935A1C3CD044219AB2009108
:10333000402A04D80320D11D814389B2009103990A
:103340001B0C8B4224D0402A22D80122300008A92D
:10335000FFF710FF021E1BD1380008A9FFF70AFF74
:103360000400042831D9009A059B9B188022520141
:10337000B218934240D288235B05C118009A09A86D
:1033800008F092FB1D4B009A09A9F01808F06CFB9D
:10339000009A029B9446634402931A4B029AFB18CC
:1033A0009A42BAD388235B05FC1821680198013939
:1033B00008F0DAFB200008F0E7FA039A07AB5A801E
:1033C00030000799FFF706FF0400002C03D100200E
:1033D00079E70428FBD988235B05E018069908F0F3
:1033E000C3FB0323EA1C9A4300D16BE7034B049908
:1033F000E01808F039FB65E70424ECE7040000114D
:10340000FFFFFF7FF80F0000F7B505001400402A0A
:1034100021D8002701AE71803780FFF7FEFE042817
:1034200016D93A003100FFF7A5FE042810D93688D6
:10343000BC420BD0BD4209D0221CB44200D9321C80
:10344000064B92B2C118280008F02EFB30B2FEBD28
:10345000C04300B2FBE703204042F8E7040000113C
:1034600037B5042204000D0001A81649FFF7CCFF70
:10347000020004280BD1019BA34208D3AB4204D025
:10348000104901A80195FFF7F9FE01203EBD0E4C41
:1034900023682000019308F077FA01992000013990
:1034A000019108F061FB80235B01E418074B9C420B
:1034B000EED10422034901A80195FFF7DFFE0020A9
:1034C000E4E7C0465555000000C007110000081190
:1034D00030B589B008F068F910226946254808F02F
:1034E0006BFB254B009A9A420ED1019B029A0F2B3F
:1034F00033D8002101240698013B08D2002900D0CE
:103500000292029B013331D10023029325E0551C26
:10351000F2D102002100EFE710341022200004A9AC
:1035200008F04AFB029B013301D1069B02938823DA
:1035300004995B05C918059B06981A03120B0491A0
:103540000592814203D02B4201D108F0ADFA019BD4
:10355000013B0193019B002BDED1029B002B03D08A
:10356000049304984168084709B030BDE025014C38
:103570002D03EFE700000111504859368022F8B5BD
:10358000964C974BD200002120001C6008F054F9A3
:103590002300944A88331A60934B1A786A23002ACE
:1035A00000D01133E3620A232365904B37221B7846
:1035B0000820A3638E4B2118E361102323628D4BF7
:1035C0003B256361C823DB00A36123008C331A60B1
:1035D0002823013AE26320646364CA67043A211D28
:1035E000CA672100BC310D602100C0310860210094
:1035F000C4310B6021000635CC310D602100083D3F
:10360000C8310D602100D0310A602200D432106030
:103610002200D832136022000227E0322100176016
:103620004222DC310A6021001B3DE4310D602100A3
:10363000E83108602100EC310B6023000521F433F0
:1036400019602300F0331A602300183290331A6097
:1036500023009433186023001E3A98331A60AF2376
:10366000DB002360644BFA262363644B644DE36004
:10367000644BF031A3642300FF31FC33B600A1603A
:1036800021611E60A5627325E5656D3D6565A565D3
:1036900096255D4AAD00E264666258606766A5667D
:1036A00000270925A767E566584F594D6067200038
:1036B0002567E2673A6015279C30676007001A208B
:1036C00038602000A0300700212038602000A8309A
:1036D00007004C4838602000F83006602600642758
:1036E000A436376026005F3FAC3637602600033FC4
:1036F000B03637602600C637B4363760260000275C
:10370000B836376038269E60424E96205E64424E40
:103710005A66DE61414E9A645E62F53EFF3E9E62ED
:103720001E269A67354A8000DE661F675F67DD6583
:103730001D661862DA67BE23394A5B00E250394BD6
:10374000D838235004302250C4225200A350C6233C
:10375000E4205B00E1500433334AE1503349344BF9
:10376000D1603449800019503349E938FF38195085
:1037700032490430195032493248D161324911631B
:10378000324951631900F4310860CE2030494000BD
:1037900011603049195019002F48F83108602F493D
:1037A000D16582212E4A89005A501A002D490832CB
:1037B000D1671A002C49B432116088212B4A890044
:1037C0005A501A002A49883211602A4ADA6407F0EE
:1037D000C3FF012008F048FAF8BDC0460004FF1FEF
:1037E0004464FF1F106FFF1F1044FF1F4A0AFF1F92
:1037F0003A07000080C3C9019A020000DC050000FE
:103800006A18000050C3000088130000F009FF1F71
:10381000204E00006509FF1F68100000C409000069
:1038200040420F0010270000FC00FF1F751CFF1F07
:103830000000FF1FC92CFF1F5130FF1FE92EFF1F83
:103840003520FF1F2527FF1F5120FF1FFD21FF1FD0
:10385000C11FFF1F4929FF1F312AFF1F8D19FF1F9D
:103860005528FF1F7925FF1F8525FF1FC11EFF1F3C
:10387000791FFF1F391EFF1F0223F0B50124624D7F
:10388000624E2B70624B91B01C70624F0393336891
:1038900000210820FB7006F049FE082006F040FDDC
:1038A0000023984205D0FA78552A02D0332A00D056
:1038B0009DE03360042006F0B3FF07F0CDFFFFF773
:1038C0005DFE07F079FF1F2201240021524B10AE4C
:1038D0001A70524B1C70524B1970524B196891431D
:1038E000163A0A431A60602219689143403A0A4323
:1038F0001A6008F0D9F908F0DFF84B4B9847C1205F
:10390000FF214A4B80001A588A431A50C522920060
:1039100098588843BF390143995098584449084002
:103920008021C9010143802099509958C00509029E
:10393000090A0143995080213E48490108F0E4F901
:10394000032322003C49019400933C4808F044F8CA
:103950002C223B4905A808F0A7F805AC617820782F
:10396000023406F0FDFCA642F8D1364C00200121BD
:1039700006F00AFE2268344B03201A40A023DB0223
:1039800013432360802322689B041343236022682F
:103990002E4B1A4080239B03134323602C4A2D4B4C
:1039A000934200D8012008F02FF907F025FF80236B
:1039B0002268DB0413432360287807F0BDFE039BD5
:1039C0001878C0B208F0C0F807F056FF224904206A
:1039D00008F0AAF806F0F0FE00F040F800F024FE2F
:1039E00000F0CCFE00F00CFA002011B0F0BD009306
:1039F0002100194A042007F0A7FF8023DB059C6201
:103A0000FFF766FD56E7C0464A0AFF1F34F0004044
:103A10001044FF1FD061FF1F480AFF1F490AFF1F04
:103A2000680AFF1FBCF00040E1A2000000E100E0D6
:103A3000FF00FFFF1444FF1F9856FF1F1454FF1F81
:103A400088BD001114F00040FF7FF8FFFFFF9FFFCB
:103A50000080FF1F106FFF1F3B000108002210B500
:103A60001100112007F0F8FF10BD0000F8B5002389
:103A70000926374F374C3B62E3681120B343E360BC
:103A800008F05AF9112008F08FF8112007F01CFFF8
:103A90004023226880251343236080236268DB0271
:103AA00013436360A3682C4A2B43A360A3680221DD
:103AB0001340A3608023A2689B0113431022A360DC
:103AC000236C072093432364236C0F3A134323642E
:103AD00080235B003B62226B204B1A402263626BA7
:103AE0001A406263A26B1A40A263E26B1340E36365
:103AF000E3681B4A1340E36006F032FC0121072013
:103B000006F042FD174B11205A6C15435D6407F017
:103B100033FFFD21144B154A89005A508023C720DA
:103B2000626B5B0313436363E36880003343E360CA
:103B30000F4B104A19581140802212020A431A50A2
:103B4000802292051A6008220B4B5A63F8BDC046CA
:103B500000F000403CF00040FFFFDFFFEFFFEFFF11
:103B6000FFFF7FFF003800400000FF1F5118FF1FBC
:103B700000E100E0FF00FFFF0000054070B5284CA9
:103B8000238C002B23D0228A002A21D1DA00238221
:103B90006382A382E38223836383A383E38322601C
:103BA0006260A260E2601F4D1F4A6420EB80934276
:103BB0000AD8FA220020D200934205D91B4A0A21D2
:103BC000981807F091FFC0B200232872238470BDBB
:103BD0000720E11CCA7F01320240CA7705D10325C4
:103BE000201DC17F01312940C17708325200A35204
:103BF000002321001A00088A01321B180231082A0A
:103C0000F9D1221DD27F9200A350626823689B18CD
:103C1000A2689B18E2689B185B099BB2C3E7C04689
:103C20001061FF1FB861FF1FB70B000030F8FFFFE6
:103C300030B503A804880B20002C0ED14968074D2D
:103C400008784978090201430A20A94205D10121D7
:103C500020001980024B1B7A137030BD192A000016
:103C6000B861FF1FF7B5150008AA16884A680F4FFC
:103C700014785278120222430A24BA4214D1012243
:103C8000DBB2019200962A0007F0E6FC041E0BD17D
:103C9000074B1B68002B07D068782A780002104376
:103CA00042425041013098472000FEBD02290000E9
:103CB0003C61FF1F30B5012503790400BFB02B42E2
:103CC00011D00A49408807F033F828420BD0084B3E
:103CD00001A95B8D4D800B80064B00221B7A60880A
:103CE0000B7104F005F93FB030BDC0463461FF1FD1
:103CF0004840FF1FB861FF1F10B50549054806F091
:103D0000CDFF0421044A054806F08AFF10BDC046D5
:103D10003461FF1FFFFF0000B4BD00114840FF1FCA
:103D200010B5024804F066FF10BDC046B53C001156
:103D3000012303700B4B1A7A4270022282709A7828
:103D4000C270DA780271032242711A7982715A794B
:103D5000C2710C2202729A794272DB7983720B2053
:103D60007047C046B861FF1F022310B50370013BC6
:103D700043700533837010330371443B43712A331E
:103D800083714433C37100230372064B04001B8804
:103D900043720A30FFF7CCFF831D0A30C0B2E370D4
:103DA00010BDC046B861FF1F10B5142007F094FE87
:103DB000124B14220021186007F03EFD002007F08E
:103DC000C3FF012007F0C8FE022007F00DFD03200D
:103DD00004F0B4F9042006F0C9F9052003F0F2FB61
:103DE000062004F0BFF8072001F0A8FA082006F02A
:103DF000F7FE092001F074F810BDC0464061FF1FB6
:103E000007F032FD012007F0DFFD07F01DFD000087
:103E1000094B10B50400984205D0012904D12000B7
:103E2000064906F03BFF10BD0229FCD1013904F020
:103E30009FFE0028F3D0F6E7FEFF00006661FF1F3B
:103E400070B50D7A100004AA2C00168810221440B8
:103E5000154220D1002E20D10A78022A18D14A68B2
:103E6000517815780E4A09022943914205D00D4A2E
:103E7000914209D01C800A2404E014220A491A80C5
:103E800007F012FE200070BD0C2208491A80F7E7E7
:103E90001C800124F6E70824F4E70B24F2E7C0466F
:103EA000F3FF0000F4FF00009C42FF1FACBE0011B6
:103EB00010B504000749084806F0F0FE074804F072
:103EC000D9FD0020E40704D50721054A054806F07E
:103ED000A7FE10BD6661FF1FFFFF0000113E00112D
:103EE000F8BD00118C40FF1F00B50C4BBFB01A7815
:103EF0000B4902A800F0FCFC6B4680B2D880002879
:103F000009D06A46074B01A91B889380064B002203
:103F1000188803F0EDFF3FB000BDC0464461FF1FAD
:103F20004561FF1FE640FF1FF041FF1F00B50C4B2E
:103F3000BFB01A780B4902A801F020FF6B4680B28F
:103F4000D880002809D06A46074B01A95B8D938071
:103F5000064B0022188803F0CBFF3FB000BDC046DF
:103F60006E61FF1F6F61FF1F8C40FF1FF041FF1F3D
:103F7000F7B50E00377A1C0008AB11003D001A8817
:103F800020231D401F423CD13378022B3BD1736864
:103F90001F785B781B023B431E4FBB4208D01E4F6D
:103FA000BB4214D01D4DAB4221D00A252800FEBDD6
:103FB000002A2AD1142C2AD82200F06807F074FDB8
:103FC000174B1C70012CF1D9FFF7B0FFEEE7002A68
:103FD0001BD1202C1BD82200F06807F065FD114B87
:103FE00004211C70104B187807F076FCDEE7E3B272
:103FF0000124009201940A00310007F02DFB050016
:10400000D4E70825D2E70125D0E70B25CEE70D251B
:10401000CCE7C046F3FF0000F4FF000002290000D7
:104020006E61FF1F4461FF1FF061FF1F332310B556
:10403000040003700A220749013007F035FD064BE2
:104040000F201B681A0AE37222731A0C1B0E62738C
:10405000A37310BDB861FF1FE061FF1F30B50125DC
:1040600003790400BFB02B4213D00B49408806F0FF
:104070005FFE28420DD06A46084B02A81B88938039
:10408000FFF7D4FF6B46D8800022608801A903F0B7
:104090002FFF3FB030BDC0466661FF1FE640FF1FE7
:1040A00010B5024804F0A6FD10BDC0465D400011E9
:1040B00070B5160004AA148805AA15784A685078C5
:1040C000117800022A4A0843801805284BD807F0C7
:1040D00073FC03131E29343F0720032C0BD8042242
:1040E000121BAA4200D92A0022491A80300009195D
:1040F00007F0DAFC002070BD0720112CFBD812223B
:10410000121BAA4200D92A001B491A80EEE7072099
:104110000E2CF0D80F22121BAA4200D92A001749F0
:104120001A80E3E70720032CE5D80422121BAA42D9
:1041300000D92A0012491A80D8E70720032CDAD8C0
:104140000422121BAA4200D92A000E491A80CDE788
:104150000720032CCFD80422121BAA4200D92A0020
:1041600009491A80C2E700220A201A80C3E7C04624
:10417000DCD5FFFF43BE00118C61FF1F33BE001171
:104180002EBE001129BE001124BE001110B50D2154
:10419000024A034806F044FD10BDC04618BE001197
:1041A000FC40FF1F13B5104C0423217C01AA00F032
:1041B000ADF9002815D16B469A88236852BA92B29D
:1041C0005343228909491B0C9B184B806B46DA88A4
:1041D000636852BA92B2534362891B0C9B188B805E
:1041E00016BD0120FCE7C046A061FF1FB861FF1F9C
:1041F00013B5124C06236A46217C00F087F900288B
:1042000019D16B461988236849BA89B24B43218971
:104210000B4A1B0C5B1853806B46D97803335B78D1
:104220001B020B435BBA61689BB24B4361891B0C59
:104230005B18938016BD0120FCE7C046A061FF1FFC
:10424000B861FF1F37B5174C07236A46217C00F081
:104250005DF9002824D16B461B787F2B20D86B4654
:10426000DD78F0232A041B031A406B469B880E4915
:104270005BBA9BB21A4323682D09534322891B0C56
:104280009B184B806B465A789B7812031B011A438C
:1042900063682A43534362891B0C9B188B803EBD85
:1042A0000120FCE7A061FF1FB861FF1F7FB5022658
:1042B000154C0022217C03AB0096050000F0F8F8B5
:1042C000002802D0012004B070BD0E23217C012201
:1042D000280000966B4400F0EBF80028F2D16B4602
:1042E0009A892368D2BA5343228908491B149B1820
:1042F0004B806B46DA89636852BA92B25343628943
:104300001B0C9B188B80DEE7A061FF1FB861FF1FAD
:1043100070B5184C237C002B0FD0382B0ED1164DC6
:10432000280000F073F8CC23AC222800217C9B01EC
:1043300000F027F9280000F0A7F870BDE3890F4AC4
:10434000934209D10C4D280000F060F800222800AB
:10435000217C00F005F9EDE7094A9342EDD1064DC5
:10436000280000F053F890222800217C920100F0F0
:1043700026F9DFE7A061FF1FD441FF1F830500007E
:104380008320000070B5144C237C002B1FD0636980
:10439000002B1CD0114D280000F038F8636928006C
:1043A00098470400280000F06FF8002C10D10C4B47
:1043B0000422995E002905DA9C801A8801321A804D
:1043C000200070BD074A9142F7DD9A80F5E701248D
:1043D000FEF78EFEF4E7C046A061FF1FD441FF1F29
:1043E000B861FF1F0F27000010B58024064AA40003
:1043F0001168436B234205D113685B1A032BF8D96C
:10440000012010BD0020FCE76008FF1F70B5C179D6
:1044100005000C00631E9C411A4BE402E41849009D
:104420000460C9B2007906F0E5F8E97968794900D5
:104430000131C9B206F0DEF8E8790930C0B207F000
:1044400043FA0023E36661332360AA795B3B002AC9
:104450000ED022689A43023B134323600A23E36190
:104460000733236200232363A3630133E36370BD37
:1044700022689A4302231343236046236361063371
:10448000A361EFE70050004070B500250400036809
:10449000DD66C0790930C0B207F04EFC29002079F2
:1044A00006F044F82900607906F040F870BD00007D
:1044B000F8B51E0006AB1D78002304681700E366FC
:1044C000616007F071F901238022E3662B00276108
:1044D0005200013B08D207F057FB08200A4A116836
:1044E000002D03D12800F8BD2261F2E7236F0342BB
:1044F00003D02369013D3370013613685B1A032B27
:10450000EED90125EEE7C0466008FF1F70B51C001C
:10451000002305681600EB66696007F045F9012382
:104520008022EB6623005200013B08D207F02CFBEF
:1045300008200A4A1168002C03D1200070BD2A61AE
:10454000F2E72B6F034203D02B69013C3370013635
:1045500013685B1A032BEED90124EEE76008FF1FF6
:10456000002370B504681500E366616007F01CF96C
:104570000123E366256107F007FB2000FFF734FF06
:1045800070BD70B51D00002304681600E36661600D
:1045900007F00AF90123E36626610F33626B1A42C2
:1045A000FCD02B0A23611023626B1A42FCD0EDB2BF
:1045B000256107F0E9FA2000FFF716FF70BD002320
:1045C00070B504681500E366616007F0EDF801233B
:1045D000E3662B0A23611023626B1A42FCD0EDB212
:1045E000256107F0D1FA2000FFF7FEFE70BD70B51F
:1045F0001E00002305681400EB66696007F0D4F81C
:104600000123A619EB660F33B44205D107F0BCFABB
:104610002800FFF7E9FE70BD21782961696B194216
:10462000FCD00134F0E7000010B5084CE368002B23
:1046300008D18022064B52021B689B186360054B11
:104640001B68236007F048FBA06010BDE061FF1FFE
:10465000C8F00040CCF0004070B5184A936A916AE7
:104660009942FBD116498A689A421FD39A1A8B60E5
:10467000144B0126186893B2D202D20E4343424330
:1046800000204C681B0A1B1912029B180E4C0A686A
:104690004B60551CA3420CD8002801D04B600A6027
:1046A0000A4A136008680A4B186070BD581E821AC7
:1046B000DDE7084A30009B182A00EAE700F00040D6
:1046C000E061FF1F140AFF1F40420F00C8F00040C6
:1046D000CCF00040C0BDF0FF70B51F4C23793F2BDC
:1046E00001D93F2323711D4B22791A701878C0B26B
:1046F00007F00AF918231A491A4A0B801A4913803D
:104700000B805380A379194980200B800C21938062
:1047100001334B43164D191C0001834200D9011C83
:104720002980D1806379002B11D101336371237A01
:10473000012B01D8022323726279237A0D48534357
:104740000A21584307F0D0F90B4D286070BDA02B0B
:10475000EDD9A023EAE7C046D461FF1F480AFF1F36
:10476000EE41FF1FBC43FF1FEC41FF1FEA41FF1F4B
:10477000E841FF1F71020000C461FF1FF8B5192155
:104780000020FEF76DFE114C011E114D09D10C22C7
:10479000104BC1CBC1C4280007F04EF8FFF79CFFB7
:1047A000F8BD0C2220000C49FEF72EFE0C2802D08A
:1047B000084B43CB43C40C2228000849FEF724FED3
:1047C0000C28EBD00C220021E5E7C046D461FF1F86
:1047D000A061FF1FA0BE0011FC0C0000F50C000042
:1047E000F0B51D4C8022A544040088206946520182
:1047F000400507F029F9902212016A4413002000B5
:1048000032C832C316C816C38023144C144FA6688E
:104810009B033343A3603B6007F08EF98823A068B5
:104820005B05C01807F0B0F8002588232900802216
:10483000A0685B05C01840196944520007F014F9DC
:1048400080230135FF355B019D42EED1A6603E60BD
:10485000044B9D44F0BDC046FCEFFFFF2C43FF1FFF
:104860009808FF1F04100000F0B5040087B000286E
:1048700025D0684606F090FF1B4C022806D1062280
:104880006946200006F0D0FF002816D069460023B4
:1048900001250F262F00E25C0133100910308740FC
:1048A00038002F00324097403A0002434A610439F1
:1048B000062BEFD16846FFF793FF07B0F0BD182233
:1048C00069460A4807F0C0F86A46A300D358013386
:1048D00005D01822FF21684606F0AEFFEAE7013452
:1048E000062CF1D1E9E7C0466509FF1F0009001158
:1048F000F0B5002504000E0085B0AA4200D186E084
:104900004B1C087801934B78897837790902194351
:10491000F3783F061B040B431F4303972070657019
:10492000252800D196E033D8112813D806F02CFFA3
:1049300069002501250125012501AA00B800B10063
:104940002501250125012501250125012501250137
:1049500005011F01232800D1DEE0DB2800D02EE175
:10496000042A00D8ACE01025052A05D0551F2A00DE
:104970003800711D07F098F805223100200007F07B
:1049800093F82A003900601D07F08EF805353EE0E7
:10499000562859D010D8332800D19DE0552839D059
:1049A0002628DAD19C4B2900132218001D0006F09E
:1049B00043FFFEF79DFB5CE0712800D177E0722891
:1049C00000D180E0602800D18BE0DC28C5D1022A2C
:1049D00000D875E07378BFB26370B378A370032A10
:1049E00005D0033A390092B2F01CFEF747FC1022C2
:1049F0003900E01CFEF708FDC51C002807DA6070CE
:104A00005CE00C222000854907F04EF80C252800B8
:104A100005B0F0BD013A824D0C2A13D8002A0AD005
:104A20002800019907F040F8FFF756FE0C222800F5
:104A30007C49FEF723FC29000C22601C07F034F8A7
:104A40000D25E4E70C22EBE7754D774B2A0043CBAD
:104A500043C2E9E7013A704D0C2A11D8002A08D068
:104A60000199280007F020F80C2228006F49FEF772
:104A700005FC29001322601C07F016F81425C6E770
:104A80000C22EDE706226A49601C07F00DF80625A6
:104A9000BDE712226749601C07F006F81325B6E748
:104AA00008226549601C06F0FFFF0925AFE7717811
:104AB000F02905D8614B188801F0BCFD0225A6E756
:104AC000FF236370FAE75E4B012A03D072789A7075
:104AD0006270F3E79B78F4E72000FFF7A7FA050080
:104AE00095E7013A564B574D062A10D8002A10D0A8
:104AF000012128005970019906F0D6FF01F056F8FF
:104B000029000622601C06F0CFFF07257FE706225A
:104B1000EEE700225A70F3E7042A04D94A4D2F60C9
:104B200007F0DAF8A860FFF797FD0422039003A9C5
:104B3000601C06F0B9FF052569E7444D062ADFD958
:104B400006222800019906F06FFE0028D8D0062220
:104B50000199280006F0A8FF06223D492800FEF72B
:104B60008DFB0123364A91780B439370C8E7012AE5
:104B7000A6D07078FFF778FEA0E7012800D0ECE619
:104B8000931E344F132B06D87378002B0BD100F0F3
:104B900015F900F04BF9304B39001D78601C6A1E86
:104BA00006F082FF33E7551E2A000199380006F00F
:104BB0007BFF38002949AAB2FEF760FBE9E7DA2853
:104BC0001DD1042A00D87BE7082A15D9B379727958
:104BD0001B021343F27912041A43337A1B06134360
:104BE0003B603B68052231002000039306F05CFF28
:104BF0000422601D03A956E7FE236370F1E7DE2857
:104C000000D05DE7511E012A01D10025FFE6019881
:104C100000F0B2FFF9E7C046A061FF1FACBE001173
:104C2000D461FF1FFC0C0000A0BE0011F50C0000B9
:104C3000AC61FF1F8C61FF1F3043FF1FF041FF1F5E
:104C4000D061FF1F8D42FF1FE061FF1F6509FF1F3D
:104C5000ADAC0000D163FF1FCF63FF1FAEDE0000CD
:104C600070477047020010B5094B0A32094C92B2E6
:104C7000DA815A8298811882207802F041FB04225E
:104C8000054B012120781A7006F026FE10BDC046A3
:104C9000BA42FF1F1A64FF1F1964FF1F013870B565
:104CA000042809D806F088FE030928081200234BBF
:104CB0000221187806F010FE70BD204B08211878EC
:104CC00007F02AF800221E4B1A72F5E78022002412
:104CD0001B4B1A4D52001A8108211A682878DC7281
:104CE00006F0DAFD2100287806F096FD012000F09C
:104CF0007BFE00F05BFFDFE7104B0821187807F020
:104D00000BF81048FFF730F80F4B104A9B79002042
:104D100093800F4A13808022094B5200D8721A8167
:104D200000F062FE00F042FF0A4B9B78002BC3D0DC
:104D3000094A136006F020FFBEE7C046F061FF1F7E
:104D4000C461FF1FF941FF1FD461FF1FBC43FF1F58
:104D5000EA41FF1FD061FF1F34F0004010B5012968
:104D60000BD1082809D1054B1B78002B05D0262232
:104D7000034B04485A72FFF775FF10BDF263FF1F23
:104D8000C461FF1FC40900000300F0B50A4D8E186E
:104D9000B14202D152008018F0BD0C782F6824096E
:104DA0003C5D0F271C700C7801313C402F683C5D46
:104DB0005C700233ECE7C046E441FF1F0D22124B4A
:104DC00010B51A700C23114C11492370093A033B9A
:104DD0001048637006F068FE2D2301220E490F482B
:104DE000A371FFF7D1FF01220D49FFF7CDFF01228B
:104DF0000C49FFF7C9FF030000200B49020018709F
:104E0000FEF73CFA10BDC046EE63FF1FCF63FF1FE5
:104E100043BE0011D163FF1F6709FF1FD663FF1F49
:104E20006609FF1F6509FF1FAEDE000070B5134C59
:104E3000142220001249FEF7E7FA431E114D132BEE
:104E400019D8AB78002B16D0431C2B7009236B703C
:104E500000230019037028780B4B01302900C0B2E1
:104E6000187006F0F1FE297822000139C9B200203D
:104E700005F0F4FD70BDFFF7A1FFECE7D163FF1F64
:104E8000AEDE0000CF63FF1FEE63FF1F10B5114BB6
:104E90001A781870002A0ED000280BD10E4B1A7801
:104EA000062A07D85423D340DB0703D50B4B1878C9
:104EB00002F026FA10BD0028FCD0074B1B78012B0E
:104EC00002D0033B022BF5D8044B0121187806F0E1
:104ED00003FDEFE7F263FF1F1964FF1F1A64FF1F52
:104EE00070B5514E514A52493070082005F042FCCD
:104EF0000121022005F048FB022005F029FC0121D8
:104F0000002005F041FB002005F022FC00F0D2FE5D
:104F1000FEF7EEF806F020FF032246494648FFF769
:104F200033FF2D24030004221C7044490130FFF795
:104F30002BFF30230470424D424C437083702E3B54
:104F4000062220004049EB87FEF75EFA062813D0C0
:104F5000200006F021FC022809D00321200006F0E1
:104F60007BFE8D23E3706E3B237119336371062240
:104F700020003549FEF782F9344B1B68FC335C6432
:104F8000FFF754FF0020FFF781FF314C314A012128
:104F9000314B1278207802F075F9304A304B127894
:104FA0000021207802F06EF901222E4B1A702E4B50
:104FB000DB78552B31D12D4B3B325A722C4B2D4A7D
:104FC000AB81EA812B826A822021307806F0ACFE28
:104FD0000120404205F08EFD0120404205F02AFEEE
:104FE000FFF7D4F8FEF788FE00F0B2FC0120404243
:104FF000FEF75EFF012006F01FFEF02001F0FEFA32
:105000000121307806F068FC307802F0D5FA1A48B1
:1050100006F0B2FBFEF72AFD70BD6422174B5B79E8
:1050200053431A000A32CBE7F061FF1F614C0011B5
:105030005D4D00113043FF1F8C61FF1FAC61FF1FEE
:10504000BA42FF1F6509FF1FADAC00004464FF1F9B
:105050001A64FF1F1842FF1FF941FF1FEE63FF1F75
:10506000CF63FF1FC063FF1FD061FF1FC461FF1F1D
:10507000C4090000CE090000F261FF1FD461FF1FC8
:10508000F8B50A0020230D001A40194263D05E4B88
:105090001B78002B5CD0FFF7DFFA5C4B5C4C5D4E5D
:1050A00099686268737A8A1ADB039A4202D3616054
:1050B000FEF7DCFC327A217A531EDBB2994205D12D
:1050C000FFF726F9002000F0A7FD15E09142F9D383
:1050D00000272772FFF756F9A37ABB4202D0A772C6
:1050E000FEF74CFD012000F097FD4B4F3800FEF716
:1050F0003BFE390006F0C8FB637A002B25D0013B4C
:10510000DBB26372002B20D1444BDB78552B01D1ED
:1051100006F032FDE37A002B12D00023A27AE3726C
:105120009A4202D0A372FEF729FD3D4A3A4F1388F6
:10513000380001331380FEF717FE390006F0A4FB98
:10514000642370795843FFF78DFD237A013323726E
:1051500020206840F8BD0BB2002B0ADA314B1878DA
:1051600006F0B2FD002801D006F01EFC80200002EF
:10517000EFE70224214206D0254B01201A72FFF7E7
:1051800085FE2000E5E70B071ED5FFF765FA1F4BEC
:105190001F49204C98684A68637A821ADB039A4256
:1051A00002D34860FEF762FCFFF7ECF8FFF7B0F8B7
:1051B000012000F031FD00F0E5FB2368DB0701D59D
:1051C000FEF76EFF0820C4E7CB0609D5FEF7D6FC34
:1051D0000D4B1B78002B01D1FEF7A2FD1020B8E784
:1051E0000124214207D0104800F06CF806F084FB3F
:1051F00000F0F8FCC5E70424080020402142A9D0B3
:10520000FEF772FEBDE7C046F263FF1FE061FF1FBD
:10521000C461FF1FD461FF1FF941FF1FD061FF1F51
:10522000B861FF1FF061FF1FDC41FF1FF0B51B4B92
:105230001B4F1B883A8804001A4E1B4D85B09A42BA
:105240000DD832889A420AD3184B1A882B889A4272
:1052500005D1174A174B12881B889A421BD005208C
:1052600001F022FA3B8802AA138033880190538010
:105270002B88114D93800F4B02A91B88D3800F4BB5
:105280002A78188802F03EFF0D4B08212878019AF1
:105290001C7006F069FB05B0F0BDC046BE63FF1F81
:1052A000EE41FF1FEC41FF1FEA41FF1FBC63FF1FE0
:1052B000BA63FF1FE841FF1F1A64FF1FF041FF1F81
:1052C000B863FF1F13B50C4B1C78002C11D10028BC
:1052D00001D00A4B18600A4A0A4B11780A4A107822
:1052E0000A4A01920A4A0092002205F0AFFA200011
:1052F00016BD1124FBE7C0461964FF1FB463FF1FEE
:105300001864FF1F0864FF1F1A64FF1FF463FF1F68
:10531000F863FF1F10B5064B12201B78052B06D132
:10532000044B13221988044B187801F099FB10BD27
:105330001964FF1FF041FF1F1A64FF1F10B50024FE
:105340000122114B52421870104B1C70104B1A80E6
:1053500002F032F904220F4B21001A700E480C3271
:1053600006F0A2FA102221000C4806F09DFA07224E
:105370000B4B1C600B4B1C700B4B1C700B4B1A70B7
:105380000B4B1C7010BDC0461A64FF1F1964FF1F31
:10539000F041FF1F1864FF1F0864FF1FF863FF1F21
:1053A000F463FF1FCE63FF1FCD63FF1FF241FF1F9A
:1053B000CC63FF1FF8B5174C0600257806A8142407
:1053C0000078052D23D1B41F134FA5B21824BD4278
:1053D0001DD88D1FADB2BD4219D8FA256D00AA4265
:1053E00015D21D000D4F0A3DADB2BD420FD80C4C79
:1053F00026800C4C21800C4900240A800B4A138023
:10540000FFF714FF0A4B0421187806F085FC2000F2
:10541000F8BDC0461964FF1F790C0000750C000030
:10542000EE41FF1FEC41FF1FEA41FF1FE841FF1F54
:105430001A64FF1FF0B50BB20D0089B0002B00DB22
:1054400070E1A44E307806F03FFC041E50D0037883
:10545000A22B00D122E1D02B1AD0912B45D1437839
:105460000E2B42D19C4B82889A423ED19B4A836844
:105470001278052A39D1032018567F2835D0984B49
:105480001B68002B31D05B68002B2ED098472CE096
:105490008078072829D806F08FFA0428183F3F742F
:1054A000A8D86378002B0CD101218C4B19708D4B3F
:1054B0001A78002A5BD08C4B307801F0E3FE00288C
:1054C00055D00722854B1A7051E061780029F8D138
:1054D000E378002B11D0854A854B1278307801F0A3
:1054E000D1FE60706378002BEBD1200006F05CFAEF
:1054F00080200002684009B0F0BD784B1B78022B79
:10550000F3D00121307806F0F7FA0028EAD1012122
:10551000307806F0E1F9E5E76378002BD1D16F4FE1
:10552000032807D13B78052B02D101333B701EE0E5
:105530000223FBE76F4B1A886F4B0293002A0BD0B4
:105540001B78002B03D00121307806F00DFA3B7850
:10555000062B04D1013BE9E7029B1A70F7E7042B05
:1055600041D10121029B3078197006F0B5F95C4BEE
:105570001B68002BB9D01B68002BB6D0574A107897
:1055800084E76378554F002B27D10622211D5B4805
:1055900006F08AFA62895A4B5A491A80A2895A4BF4
:1055A0001A80E3890B800521397058490A80584ACE
:1055B0001380228A574B1A80574B1B78012B09D135
:1055C0001F2001F071F8FA22920042430421307842
:1055D00006F0CAF90022484B75E7312B00D070E77E
:1055E0000022454B1A700323A0E7062200214348FE
:1055F00006F05AF90023454A04211380444A3078C2
:105600001380444A138006F087FB0821307806F0A7
:1056100083FBA379083B5A425341304A033313704A
:10562000304B1B78002B06D0334B30781A78002A89
:1056300006D001F065FE0122314B52421A8096E7F6
:105640000121197006F048F9F5E70821307806F0D5
:1056500063FB6378002B00D047E72C4B2D4F029360
:10566000E388029A04211380294B3078039323891D
:10567000039A138063893B8006F03EFA002800D02D
:1056800033E7264B1B68002B00D12EE703990298C5
:105690003A88098800881B68984726E74379132BC6
:1056A00000D022E70389012B0AD11D4B1B78022B66
:1056B00006D10821307806F02FFBFFF72BFE14E708
:1056C000052000F0F1FF08210200307806F04CF9C7
:1056D0000BE7C0461A64FF1F051400001964FF1F82
:1056E000B463FF1F1842FF1FF941FF1FEE63FF1F46
:1056F000CF63FF1FF063FF1FF263FF1FC163FF1F34
:10570000F041FF1FC863FF1FCA63FF1FBE63FF1F77
:10571000BC63FF1FBA63FF1FC063FF1FB063FF1F9F
:10572000B863FF1F8020C001014200D0E2E6CB0732
:1057300031D5324B1B78002B1DD0314E05AC337860
:10574000052B1AD1023B23702E4B21001B782372AC
:105750002D4B1B7863722D4B187801F037FD002814
:1057600009D007202A4B30701B68002B03D01B6820
:10577000002B00D098470120BCE60E20254B0622C6
:105780001B7825492370254B1B78637002ABC0182A
:1057900006F08AF9D8E7022308001840194209D018
:1057A000174B1B78052B03D11D4B188806F074FA94
:1057B00002209FE60424214203D0FFF737FD20009A
:1057C00098E6082308001840194200D193E6154BCB
:1057D0001C78012C03D0022C0DD008208AE6124B35
:1057E000124A134913481B881288098800880094BC
:1057F000FFF7E0FDF1E7FFF78DFDEEE7F263FF1F36
:105800001964FF1FF241FF1FCC63FF1F1A64FF1FC3
:10581000B463FF1FCE63FF1FF341FF1FCD63FF1F64
:10582000F041FF1FB863FF1FE841FF1FEA41FF1F60
:10583000EC41FF1FEE41FF1F10B502A804880B20AA
:10584000002C10D1496808784978090201430C48B6
:10585000814209D1022119800A4B59881170DB78E5
:1058600000205BB2537010BD074C0A20A142FAD150
:1058700002211980034B998811705B79F0E7C046CB
:105880006E2A0000B861FF1F6F2A0000F7B51500EF
:1058900008AA16884A680F4F1478527812022243D9
:1058A0000A24BA4214D10122DBB2019200962A00E6
:1058B00005F0D2FE041E0BD1074B1B68002B07D04E
:1058C00068782A78000210434242504101309847DC
:1058D0002000FEBD022900002C64FF1F30B5012509
:1058E00003790400BFB02B4225D01449408805F04D
:1058F0001FFA28420CD0124B01A95B8D00220B80AD
:1059000002234B800F4B5B888B80608802F0F0FA9B
:105910000D49608805F00CFAC0070CD50B4B01A9A6
:105920001B8800220B8002234B80064B9B888B80B8
:10593000608802F0DDFA3FB030BDC0462464FF1F2E
:105940001C42FF1FB861FF1F1C64FF1F7642FF1F30
:1059500010B5074C0749200005F0A0F920000649C2
:1059600005F09CF90721054A054805F059F910BDD5
:10597000FFFF00002464FF1F1C64FF1FCCBE00114A
:105980001C42FF1F10B5024803F034F910BDC04699
:10599000DD58001170B55F25082607498400CA78D4
:1059A0008B7840012A40B3433440A8432343024349
:1059B0008B70CA7070BDC0468D42FF1F010043B29C
:1059C00004205A0002409B000C3003401A43152368
:1059D00010B5044CE0789843143B0B401843024345
:1059E000E27010BD8D42FF1F10B5054B08241979D8
:1059F0000A00A243002801D022000A431A7110BDF8
:105A00008D42FF1F10B5054B4024D9780A00A243F0
:105A1000002801D022000A43DA7010BD8D42FF1F1A
:105A20000821F8B5324D334BAE7804000E40AE700D
:105A3000984204DD67232B70473B6B70F8BD2E4BFB
:105A4000984203DAE0232B703A3BF6E700232B70F1
:105A50006B7083B21A0029485F3292B2284F82429B
:105A60002CD9002C03DA5B421CB204232B700534C2
:105A700020B20A2106F038F804B2FA239B009C42B7
:105A800032DB08232A7813432B706421200006F0B0
:105A90002BF80A2100B206F067F909B22A787B5C7C
:105AA00013432B700A21200006F01EF80A2100B2D1
:105AB00006F05AF909B27B5C6A780AE06970002C3A
:105AC000DBDA5B421CB204232B70F3226B78092CC7
:105AD000E8DC13436B700A21200006F045F909B297
:105AE0007B5C1E43AE70A9E7632CCEDCEDE7C046BD
:105AF0008D42FF1F1B4E00001DFCFFFF2A08000007
:105B0000F6BE00110823F7B5194FCD003E79040009
:105B10001E403E71EDB2632806DD5F3333433B71B7
:105B200020231D437D71F7BD0300093305DA2023CF
:105B30005B4233433B71A623F3E70E4B01930028EE
:105B40000BDA0423444224B23B710A21200006F000
:105B50000BF9019B09B25B5CE3E70928F5DD0A213B
:105B600005F0C2FF019B00B21B5C1E433E71ECE7D7
:105B70008D42FF1FF6BE0011F8B50A4F05003B78B5
:105B80000E00002B0CD0084C2000FEF73FFC330029
:105B90002A0020003978FEF72AFD2000FEF774FC69
:105BA000F8BDC0463764FF1F9442FF1F70B50A4E10
:105BB0000A4D06223100280005F036FE002809D0E3
:105BC000074C31000622280005F06EFF0721200057
:105BD000FFF7D2FF70BDC0468D42FF1F3164FF1F2B
:105BE0003064FF1FE622402110B50A4B1A70403A7C
:105BF0005A703E329A70DA780A40DA7008221979BF
:105C00001140053A0A431A71D7225A71FFF7CEFFA5
:105C100010BDC0468D42FF1F10B5002838D0214C62
:105C20000223E05E204B1B685B0632D5092332213C
:105C3000584305F059FF4130FF3000B2FFF7F0FE46
:105C40000520FFF7A7FE0422A35E184A63209342B3
:105C500005DC32331800642105F046FF00B2012153
:105C6000FFF750FF237A0024132220009A4260415C
:105C7000C0B2FFF7C7FE2000FFF7A0FE0C4B18785C
:105C8000053843425841C0B2FFF7AEFEFFF78EFF22
:105C900010BD0A21053005F027FF00B2FFF7C0FE56
:105CA0000320CEE7B861FF1FD461FF1FDD2600008F
:105CB0001964FF1F70B500250A4C2000A571FEF77E
:105CC000A5FB10233E212000074AFEF790FCA842C6
:105CD00000D13E35054B20001D70FEF7D5FB01239A
:105CE000A37170BD9442FF1FE6BE00113764FF1F11
:105CF0000200F0B501270A480A4E51188B1A002BF2
:105D000000DCF0BD082415784308684038404000A6
:105D1000805B013C58406D08002CF5D10132EDE765
:105D2000FFFF000006BF0011F0B500250F269D42C1
:105D300000DBF0BD4C5D070944403440A400A0588E
:105D400001357840F3E70000F0B589B06A460D00F0
:105D50000B000F27110010351C7801332600240991
:105D60003E40167054700232AB42F5D12023024AF5
:105D7000FFF7DAFF09B0F0BD0CBF0011F0B54E78A7
:105D80000B7889B036020C00170001901E43012ADF
:105D900061D9954B9E4200D877E001339E421CD1D9
:105DA000062A17D1CA788B7812021A430B791B0482
:105DB00013434A7912061A438C4B5A6100221A7017
:105DC0005A808B4A5A608B4A9A608B4ADA6000206C
:105DD00009B0F0BD88225205EEE7884B9E423CD1C7
:105DE00082498B78002B00D0F6E00C2A31D10F22AB
:105DF000A3789343E27812021343227912041343E7
:105E00006279120613434B60E279A07912020243D1
:105E1000207A00041043627A12060243CA60E27AD2
:105E2000A07A1202024376484A81834208D80423AA
:105E30006E49142201980B7005F036FE1420C7E756
:105E40001201D21889235B059A42F0D801238B7086
:105E5000BDE7022AFAD00523EAE76A4A01239642FF
:105E6000E6D1FFF757FA052F0CD9E378A2781B0289
:105E70001343227912041A4363791B061343624ABF
:105E80000393136005F078FEA1E7584D2B78002BA3
:105E90009DD1AB78002B00D1A0E02B8901339BB2C0
:105EA0000093B34200D091E0132AD4D9CF7C8B7CED
:105EB0003F02122120001F43FFF71AFF874200D044
:105EC0008EE0002E3DD1E378A2781B0213432279A5
:105ED000E96812041A4363791B06134303930A22E9
:105EE0008B4212D1FF23A370E370237163716B891E
:105EF000002B09D1E37B227C1B0212041343A27BFB
:105F000013431B0901336B8100226B89002B8ED058
:105F1000002A67D1686837013818000B6B690003E5
:105F20000390984205D9686105F02EFDEB780133A6
:105F3000EB7068681022A11C381805F095FD2E81C1
:105F400045E76F89009A7B1E9BB293423AD1E27873
:105F5000A37812021A43237905A81B04134362791C
:105F60006C6812061A43EB6800920392211D0C2202
:105F7000049305F099FD0120260004A94042103643
:105F8000FFF7E2FE013F012F17D1009A0B23286192
:105F9000824200D04CE704221C49200005F064FD39
:105FA000042203A9686805F04FFDE968039AFF23FE
:105FB000914200D13CE7F73B3AE73100FFF7C4FEDE
:105FC0001036DFE70923B742A4D831E7009BB3427C
:105FD00000D9FCE607232BE7022329E7032327E761
:105FE000062325E70A2323E7FFFE00009C42FF1F4C
:105FF00000000111FFFF00005048593601FF00006A
:10600000FFFF001102FF000034F00040A842FF1F14
:1060100010B5034C0B000122210000F06BFA10BDFB
:10602000D16100110B8870B506000D000224162BFB
:1060300011D92B000322094900F05CFA041E0AD191
:10604000074B2A881B88191C934200D9111C300069
:1060500089B200F0EFFA200070BDC046FD6100116A
:106060004A64FF1F10B54A780400013A0B00022071
:10607000012A07D80A78002A04D005222000024904
:1060800000F038FA10BDC0462B6200110A7810B536
:106090000B0004000220002A04D00722200002493D
:1060A00000F028FA10BDC046D76200110A7810B57A
:1060B0000B0004000220002A04D00922200002491B
:1060C00000F018FA10BDC0463D63001110B5034C36
:1060D0000B000B22210000F00DFA10BD6D630011C2
:1060E00010B5034C0B000D22210000F003FA10BD87
:1060F000DF63001110B5034C0B000F22210000F0EC
:10610000F9F910BD396400110A7810B50B000400CC
:106110000220002A04D011222000024900F0EAF9EE
:1061200010BDC04649640011002310B513221900A8
:1061300000F0E0F910BD000010B5034C0B00172271
:10614000210000F0D7F910BD9B640011002310B5A9
:106150001922190000F0CEF910BD000010B5034C53
:106160000B001B22210000F0C5F910BDD564001101
:10617000F7B584890D0006000121002C22D00023F0
:106180008268D3561778002B1EDA0C2C1AD90C3CD7
:10619000A4B2131940880093230002F086FE431E28
:1061A000984101307B06DB0F6B703F23013C1F40A1
:1061B000A4B22870AF70AC80002C07D0B368013354
:1061C000AB6000210800FEBD0020EBE7AC60F8E703
:1061D0000B7803704B8843704B881B0A83700B79D4
:1061E000C370042070470420022B06D1002053788E
:1061F00011781B02009A0B43138070470B880370C1
:106200000B881B0A437002207047042000998342C8
:106210000AD1537810781B0203430B80D37890780F
:106220001B02034300204B807047F8B50D004B78EC
:1062300001240021461C03702B788B4201D82000DA
:10624000F8BD6B78B01C4F1C012B10D18900691868
:106250004B88022233704B88B9001B0A737069188F
:1062600005F0EAFB04360434A4B2F9B2E4E71223E1
:1062700059436B185A88043132705B8810221B0A0C
:106280007370691805F0D8FB12361234ECE770B55C
:10629000049D14001E00052B01D8042070BD6378F6
:1062A00012781B0213432B80E378A2781B0213435E
:1062B00002226B802A71211D681D063E05F0BCFB81
:1062C000B2B22A81E92AE8D82800A11D0A3005F0D7
:1062D000B3FB0020E2E7002310B50A789A4201D808
:1062E000900010BD9A008A185488013304705488B5
:1062F000DBB2240A4470948884709288120AC270B7
:106300000430EAE710B51100029C062B04D00420EB
:106310001022142B01D010BD022222714B78087874
:106320001B0203432380CB7888781B0203436380DE
:106330000431601D05F080FB0020ECE710B50C78FF
:106340008B7804315C43E4B203702200013005F025
:1063500073FB601C10BD0420022B06D10020537873
:1063600011781B02009A0B431380704710B50C0084
:106370000A88023105F060FB208810BD70B504006A
:106380000D0004981100012B01D8042070BD16786F
:1063900052781202324302800200F13255701470BA
:1063A000E125002C00D10C35023B9AB24280AA4272
:1063B000EBD80231043005F03FFB0020E6E7042073
:1063C000009983420AD1537810781B0203430B8053
:1063D000D37890781B02034300204B80704710B5A0
:1063E0000C000A88023105F027FB208810BD000050
:1063F00070B501211E000420049C0E400B4218D1F0
:10640000CB40DDB28D4214D90A49DBB209889942EA
:106410000FD32300EE331D70330058001118497854
:10642000165C0902314301332152D9B28D42F4D8AE
:10643000002070BDB442FF1F10B50C000A88023165
:1064400005F0FAFA208810BD10B50C788B7804316D
:106450005C43E4B203702200013005F0EDFA601CE9
:1064600010BD10B511000298032B01D8042010BDF7
:1064700014785278043B120222430280CA788C7846
:106480001202224342809AB28280EB2AEED8043173
:10649000063005F0D1FA0020E9E710B50C000B88B2
:1064A00003700B881B0A43704B8883704B881B0A50
:1064B000C3708A880430063105F0BEFAA088043023
:1064C00080B210BD0420012B03D100201378009A64
:1064D0001370704710B50C000B8803700B881B0AF3
:1064E00043704A880230043105F0A6FA6088023011
:1064F00080B210BDF0B589B003931E4B02924200EA
:106500000700D05A019102F020F81325061E2DD065
:10651000029B01240370019B002B04D000190399F6
:106520009847001984B26B461B7A5BB2002B0FDAD6
:106530001021380002F01CFB1925002813D130006F
:106540003219E1B202F066FC051E0CD10C34A4B283
:10655000042304AA380005A993800696948101F0CB
:10656000AFFD051E02D0300005F0E6F9280009B0A5
:10657000F0BDC0464864FF1F70B505000C00002840
:106580000CD00020814209D010222000044905F0DF
:1065900053FA01202B7823736B78637370BDC04668
:1065A0004CBF0011F0B506000D0017001C0085B0AF
:1065B00002291BD00020102907D1022B07D0102B55
:1065C00003D115E00020102C08D005B0F0BD6946BD
:1065D0003800FFF7D1FF2A0069460BE0694630001A
:1065E000FFF7CAFF22006946380004E0022BE9D118
:1065F0002A003900300005F00FFBE6E7031CF02805
:1066000000D9F023032008499AB2013A0B80D3172E
:10661000034006499B189B100B80D30F04499B181D
:106620005B100B807047C046B842FF1FB642FF1F89
:10663000B442FF1F034B1B888B4202D3024B400026
:10664000C1527047B842FF1F4864FF1F014B400012
:10665000185A70474864FF1F1722014B1A80704771
:106660004864FF1F70B505000E2005F095F9041E63
:1066700013D0D0230370002306228370074945708E
:10668000033005F0D9F9064B2100DA8A62811B7EBE
:106690002373044B187805F0A7F970BD6464FF1FDD
:1066A0005464FF1F0843FF1F262803D8024B4000F5
:1066B000C05A70470148FCE7BA42FF1FFFFF0000C5
:1066C00070B506000C00094D1C220021280005F0C1
:1066D000EBF8074B1E70074B1C7005F0EDFA012319
:1066E000002801D0002312202B7070BD5464FF1FBE
:1066F0000843FF1F7564FF1F70B505000D4C0800AF
:10670000E260A16010220021656005F045FA0128D1
:1067100003D11021A06802F058FD102200212800AA
:1067200005F03AFA012803D11021606802F04DFD0E
:1067300070BDC0465464FF1F70B5041E05D100290A
:1067400003D006220D4805F077F90D4B1D78012D79
:1067500011D1002C05D102221A7005F04DFA280043
:1067600070BD00221A70074B1B78FF2BF7D020005A
:10677000FFF778FFF3E70025F1E7C0466464FF1FE9
:106780005464FF1F0843FF1F030010B5002801D108
:10679000002010BD00780B4A002803D15988D1820F
:1067A0001B7913761378022BF2D10023984200D183
:1067B00003331370044B1B78FF2B01D0FFF752FFFC
:1067C0000120E6E75464FF1F0843FF1F002911D092
:1067D00000280CD04B79012803D1402252421343A8
:1067E00003E03F221340032802D001204B71704781
:1067F0004022F4E70800FAE770B5094D0100287857
:1068000000280BD0074C0622200005F015F92100C6
:106810002878FFF7DBFF200005F006FA70BDC046C0
:106820007464FF1F4E64FF1F00290AD0012808D19D
:106830003F224B799343C02B03D0403B5A425341F4
:10684000981C704770B5174D06002B78FF2B15D09C
:106850000A2005F0A1F8041E10D0D0230370C83B15
:106860008370114B11491B784670C37006220430A7
:1068700005F0E2F82100287805F0B6F80C4B1B78FB
:10688000012B0DD10B4B1B68002B03D09B68002BF9
:1068900000D09847084B04211878084A04F0FCFF00
:1068A00070BDC0460843FF1F7464FF1F4E64FF1F86
:1068B0007064FF1F9C64FF1FA064FF1F60EA00005C
:1068C000014B98687047C0465464FF1F014BDB685A
:1068D000186870475464FF1F074B10B5DA681368D7
:1068E00001331360054B1878FF2803D08021C901BC
:1068F00004F0F2FF10BDC0465464FF1F0843FF1FA1
:10690000F7B50E0002F0C8F8051E1CD00E4B06624B
:106910001F78002F00D10778AB791020019305F084
:106920003BF8041E0FD0D0230380C73B8370019B2C
:10693000E91DC3700622043005F07EF821003800FE
:10694000E66005F051F8F7BD0643FF1F014B1878CC
:106950007047C0467464FF1F054B002805D1054BE6
:106960001A78054B002A00D1014B18007047C04629
:106970006464FF1F7464FF1F4E64FF1F014B58685F
:106980007047C0465464FF1F024B1868431E98416D
:10699000C0B270477864FF1F421E03000120152A11
:1069A00003D9FF3B5A425341D8B27047F0B51C009F
:1069B00000230E0085B0039002920B70029A93425E
:1069C00001D3002019E0E55C5A1CD2B2002DF8D0AA
:1069D000029851198142F4DC0233DFB2A35C180043
:1069E0000193FFF7D9FF002807D0013D019A0399D1
:1069F000EBB233708A4202D1E01905B0F0BDDB1969
:106A0000DBB2DBE710B50C0002F09EF803001220A9
:106A1000002B03D02100588804F0D6FE10BD0000E2
:106A200070B50E4D84006359002B15D0186A0028EC
:106A300001D004F059FF2B59586A002801D004F006
:106A400053FF2B59986A002801D004F04DFF2859B4
:106A500004F04AFF00232B5170BDC0468464FF1F21
:106A60001C4B70B504000E00150099420AD11A4B58
:106A70001B68002B01D1122070BD1B68002BFAD0BF
:106A80009847F9E7154B994215D1134B1B68002B1A
:106A90000AD01B68002B07D09847002804D1104B60
:106AA0001C70104B1D70E7E729002000FFF7AAFFBC
:106AB0000028E1D1F3E7080001F0EEFF0028DAD06A
:106AC00003780320A342D7D12900300004F07CFED4
:106AD000D2E7C046FEFF00008064FF1FFFFF0000FA
:106AE0007D64FF1F7C64FF1FF7B50400808801F000
:106AF000D3FF0025A84203D00578A08802F008F84B
:106B00001C4E3378002B1FD0AB421DD11A4B2800EE
:106B10001978FFF777FF002818D000233370A37986
:106B20000820A778A688019304F036FF011E0DD037
:106B3000D0230370CA3B8370019B477086808371AA
:106B4000280004F051FF01E0002DE8D1A0880B4B94
:106B50008200D358002B01D0FFF762FF1721A088D5
:106B6000FFF768FDA08801F027FDA08801F0FEFD79
:106B7000F7BDC0467D64FF1F7C64FF1F8464FF1F58
:106B8000F0B587B01D000CAB1B88070001930DAB5F
:106B90001B88142002930EAB1B88160003930FABC7
:106BA0001B880091049310AB1B88059304F0F4FE3E
:106BB000041E1AD0D0230370CB3B47708370C6707D
:106BC000062229000430002D11D004F035FF019B6E
:106BD00021006381029B0098A381039BE381049BB6
:106BE0002382059BA37404F0FFFE07B0F0BD04F000
:106BF0005BFEECE7F7B5009308AB1B8807000C20A1
:106C00000D001600019304F0C7FE041E13D02800E7
:106C100001F042FF00280FD00078D0232370C93B39
:106C2000A370009B21002381019B6770A580E680F3
:106C3000638104F0D9FEF7BD014B1878EDE7C0463B
:106C40000843FF1F13B5040064890389C288818843
:106C5000C0780094FFF7CEFF13BD000010B5044CC0
:106C60002068002803D004F03FFE0023236010BDFD
:106C70008864FF1FA122F0B5818892004A43384BF7
:106C8000384F1B6804009B189D2292009B18827944
:106C900089B01A603B68002B5FD01D78324B1B68AF
:106CA000002B04D05B68002B01D000209847260001
:106CB00008363100E079FFF7B7FD237DE07102006F
:106CC000E0780493638A29000393238A0293E3897B
:106CD0000193A38800933300FFF752FFE378002B62
:106CE0000BD1E289A379A18802920196E27928006A
:106CF0000092012201F0DAFEE0703B68002B20D008
:106D0000FFF7ACFF194D287800281AD0184B1978D6
:106D1000FFF778FE002814D02B78E6780820079338
:106D2000A78804F039FE011E09D0D0230370CA3BA6
:106D30004670837087808671079804F055FE0023A3
:106D40002B701721A088FFF775FCA08801F034FC98
:106D5000A08801F00BFD09B0F0BD064B9DE7C046D1
:106D60003409FF1F8864FF1F9C64FF1F7D64FF1FA1
:106D70007C64FF1F0843FF1FF8B5070008000E00E2
:106D800001F08AFE041E18D02620FFF78DFC051E98
:106D900000D12578062004F0FFFD041E0DD000214F
:106DA000062204F081FDD0232370C23B21006770CE
:106DB000A370A680E8B204F017FEF8BDF0B585B068
:106DC00001930AAB1B78070002930BAB1B780800FA
:106DD0000D000092039301F05FFE061E22D01020EA
:106DE00004F0DAFD041E1DD01022002104F05CFD29
:106DF0002620FFF759FC002800D13078D0232370DB
:106E0000C13BA370009B21002372019B67706372DA
:106E1000029BA580A372039BC0B2E3720C9BE3604C
:106E200004F0E2FD05B0F0BDF7B50D00019001F0F2
:106E300033FE071E20D00E2004F0AEFD041E1BD032
:106E40002620FFF731FC061E00D13E78D023238098
:106E5000C53B0622A370F91DE01C04F0EDFD019B6B
:106E60002A0063810123DD401A401D402100227366
:106E70006573F0B204F0B8FDF7BD0000F0B585B061
:106E8000029010000D0017000A9E039301F004FE0B
:106E9000041E31D0029B002B2ED1039B02795B078D
:106EA00024D5122313430422002E08D10B99002964
:106EB00005D10C99002902D10D9900291AD01A4345
:106EC0000D9B2271002B00D0C9E0002E00D1CFE035
:106ED000002D00D0CCE0606A002801D004F004FD51
:106EE0001C21300004F020FC606205E002239A437C
:106EF0000E33D7E793432371654BBA00D458002C67
:106F000000D1AAE0002E10D0236A002B03D11C2050
:106F100004F0E2FD20625E4BBA00D358186A0028E4
:106F200003D01C22310004F087FD0C9B002B12D0F3
:106F3000574CBB001D596B6A002B03D1162004F07F
:106F4000CBFD6862BB00E358586A002803D01622C4
:106F50000C9904F071FD0D9B002B11D04C4DBC0021
:106F60006659B36A002B03D1142004F0B5FDB0625A
:106F70002B59986A002803D014220D9904F05CFD67
:106F8000380001F089FD051E67D0414BBA00D35887
:106F9000002B62D01A6A3420002A00D11C389A6A69
:106FA000002A01D0143080B20B9A002A01D01C3084
:106FB00080B25B6A002B01D0163080B204F0ECFC8A
:106FC000041E4AD01822002104F06EFC2620FFF790
:106FD0006BFB0190002801D12B780193D023237003
:106FE000029B200063700A23294EA370039BBD00FF
:106FF000A371AB59A780196A1830002905D01C224B
:10700000A06004F019FD200034307359996A0029FA
:1070100007D0030014221433E060029304F00CFD47
:1070200002980B9B002B08D003001C221C330B99E9
:107030002061029304F000FD02987359596A0029F7
:1070400003D01622606104F0F7FC6B46210018792A
:1070500004F0CAFC3800FFF7E3FC05B0F0BD1022D5
:107060000D9B0D991B69A018236204F0E5FC2CE729
:107070000B9B002B00D13FE7012D00D03CE7606A5D
:10708000002801D004F030FC1C210B982AE7C046F0
:107090008464FF1F10B5044C2068002803D004F05E
:1070A00023FC0023236010BD7864FF1F0B4B07B542
:1070B0001A68002A01D100200EBD6946531C012028
:1070C00012780731FFF772FC0028F4D00278012310
:1070D000100018401A42EED0EEE7C0469464FF1F3D
:1070E000F0B51F4F01203B6887B0002B25D09B785F
:1070F000059300F0B3FB002821D00A20FFF7D4FA53
:1071000004000B20FFF7D0FA164B05001E78731E03
:107110009E413B68F6B2191DD878FFF757FB3B68D4
:107120002900DA7A043303929A790193029200904B
:1071300033002000059A04F017FB07B0F0BDFFF7FD
:10714000B5FF002805D00620FFF7AEFA040007209F
:10715000D8E70820FFF7A8FA04000920D2E7C046C4
:107160007864FF1F7464FF1F70B50A4E0400337803
:107170000D00FF2B0DD0042004F00EFC011E08D0E2
:10718000D0230370CE3B45708370C470307804F018
:107190002BFC70BD1843FF1F70B5040006200D00C6
:1071A00004F0FAFB011E0AD0D0230370CD3B83709C
:1071B000054B44701B688580187804F015FC002C82
:1071C00001D0FFF767FF70BD7864FF1FF8B5264F49
:1071D00006003B680D001124002B05D10522234B2E
:1071E0001B78134202D112242000F8BD204A10243B
:1071F0001268002AF8D01278002AF5D0DB0719D5DA
:107200002B789A1E012A1AD80C2004F065FC13244E
:1072100038600028E8D000230A2243702900067055
:10722000023004F009FCFFF75BFF041E0AD0FFF7F1
:1072300031FFD9E700F012FB0028E1D1E4E7002B91
:10724000E2D0D0E70B4B1B78032BCDD11D20FFF7ED
:107250002BFA094B18800028C6D0084B0421187857
:10726000074A04F019FBBFE77864FF1F7564FF1F2E
:107270009464FF1F7464FF1F7264FF1FA064FF1FEC
:1072800060EA0000F7B50193194B14001A78052342
:1072900006000F0012201A4221D0012920D1154BDF
:1072A0001D68002D1BD002201F2C18D8002C02D0E6
:1072B000019B002B13D0104B1F221E706E1C00214F
:1072C000300004F0F1FA01992200300004F0B4FB20
:1072D000310020002C70002F06D004F0F5FBFEBD1D
:1072E000064B12201D68DCE704F0AEFCF7E7C04651
:1072F0007564FF1F9464FF1F1843FF1F9064FF1FF6
:10730000F8B50F4E12243368002B17D01B780F3CB2
:10731000834213D100250B4F0221387804F0FCFC86
:10732000094B042138781D8004F0F6FC074B280037
:107330001D8033685C7004F0BFFA04002000F8BDC3
:107340007864FF1FA064FF1F8C64FF1F7264FF1F1F
:1073500070B5012823D11B4C2388002B03D01A4A77
:107360001578002D07D0194B1B68002B02D0187818
:10737000FFF7C6FF70BD3B2B02D93C3B2380F9E7EA
:10738000134E0221307804F0C7FCFA2223889200C1
:1073900002215A43307804F0E7FA2580EAE70B4BE4
:1073A0001B68002BE6D00B4B1B785B07E2D5084B24
:1073B0000221187804F0B0FC0022024B1A80FFF77B
:1073C00069FED7E78C64FF1F7064FF1F7864FF1F9E
:1073D000A064FF1F7564FF1FF8B51E4D28680028C4
:1073E00003D004F081FA00232B601B4E3068002884
:1073F00003D004F079FA00233360184F05243B785A
:1074000018002040234221D0154800F02BFA3B7889
:10741000234213D0202004F05FFB2860002813D003
:107420002022002104F040FA202004F055FB041E25
:10743000306005D02022002104F036FA002004E05C
:10744000286804F051FA2C601320F8BD00F00AFA05
:10745000F4E7C0469464FF1F9064FF1F7564FF1F2C
:107460000C43FF1F10B50A4C23681A1E0ED00028CB
:1074700008D10130587004F01FFA002805D02368A5
:10748000002B02D00021FFF787FE0122100010BD63
:107490007864FF1FF7B5274E050033680191181E69
:1074A00021D05C78244F012C30D1FFF7FFFD00285C
:1074B00025D02000FFF7F8F80400412814D91F4B0D
:1074C000022118781E4A04F0E7F91E4B3C3C1C8050
:1074D000022233685A703B78002B14D1280001999E
:1074E000FFF75AFE0120FEBDFA2292004243002A15
:1074F000EED0124B0221187804F036FAE8E7FFF7D5
:10750000D3F80200F3E700233B70EBE73B78002B56
:10751000E8D1032004F040FA011E08D0D023037004
:10752000CC3B457083703368187804F05DFAFFF740
:10753000B1FDD7E77864FF1F7064FF1FA064FF1FD1
:1075400060EA00008C64FF1F10B5174983880200B1
:107550008B4220D011D815498B4217D014490020F6
:107560005B1899B2012907D8926811785A425341A1
:10757000D8B2FFF7F9FD012010BD0E4A00209B187C
:1075800007229BB29A424041C0B2F5E7836818785F
:10759000FFF768FFF0E7836899785A78090218784E
:1075A0001143FFF777FFE7E70A20000006200000FD
:1075B000F8DFFFFFAFDFFFFF014B18707047C046D9
:1075C0001943FF1F10B5064C207001F041FA2078D6
:1075D00004F0C2F90521207800F062FD10BDC0461C
:1075E000A064FF1F0BB273B50D00002B00DBC4E0DD
:1075F000884B187804F068FB041E0ED00378912B9A
:107600000FD0A22B00D1A1E0834B1878FF2852D0D5
:10761000210004F0E9F900284DD1802000026840E3
:1076200076BD43780F2B76D013D8052B70D00E2B58
:10763000EAD18088794B98422BD8794B98421BD855
:10764000784B9842E0D1A3681878591CFFF774F87A
:1076500038E03E2BD8D18378032B74D06CD8012B23
:107660006ED0022BD0D1704B1B68002B23D05B68EF
:10767000002B20D098471EE06C4BC0180C28C3D8B4
:1076800004F03AFB1DC2C2150BC20B0B0B3223C216
:107690003C00674BC0180728B6D8664B1B68002B08
:1076A00009D01B68002B06D0200098470AE0A36889
:1076B0001878FFF7C7F8200004F076F9ADE7A06866
:1076C000FFF762F800289FD0F5E7A3681B78002B2E
:1076D000F1D0554B1B68002BEDD01B68002BEAD076
:1076E000210055489847EDE74F4B1B68002BE2D02F
:1076F0001B68002BDFD021005048F3E7504B1B687C
:10770000002BD8D05B68002BD5D021004348E9E797
:10771000FFF7EAF9CFE780884A4B984203D04A4BFB
:10772000984200D070E7464B1B68002BC3D05B68C3
:10773000002BC0D02100D5E7153B012BBBD963E757
:10774000FFF798FAB7E7FFF77DFAB4E73F4B1B78EE
:10775000042B07D100236A4613800179408800F08A
:10776000C5FCA8E7364B1B68002BA4D05B68002B38
:10777000A1D00100364898479DE7012421420AD054
:10778000294B1B68002B04D05B68002B01D0002024
:107790009847012043E78B070AD5264B1B68002B2F
:1077A00004D05B68002B01D020009847022036E708
:1077B0000421280008400D4200D131E7254E3388CE
:1077C000002B21D0013B9BB23380002B1AD1FFF755
:1077D000DBF800280AD0204B1C70164B1B68002BCE
:1077E00004D05B68002B01D020009847FFF7C6F853
:1077F000694601F001FD6846FEF7FEFF1D20FEF719
:1078000053FF308004200AE7024B187804F084FA12
:10781000F8E7C046A064FF1F1943FF1F0E200000B9
:1078200001200000091000009864FF1FFEDFFFFF29
:10783000AFDFFFFF9C64FF1F0C2000000B20000047
:107840008064FF1F0D200000132000007564FF1FDF
:10785000FFFF00007264FF1F7064FF1F10B501F08E
:107860009BF910BD014B18607047C0469C64FF1F18
:107870000B880020162B01D817230420014A1380FF
:107880007047C0464A64FF1F00207047074A030044
:107890001188814207D091880020994202D101309D
:1078A0008000101870470020FAE7C046A864FF1F48
:1078B000F0B58F7806000D00C5B01E2F15D1FFF76B
:1078C000E5FF051E03D10024200045B0F0BD0022D5
:1078D0003B003100C078009200F0B2FB0400A81C0D
:1078E00000F0D2FBFF23EB70EEE7264B0624039358
:1078F0001B78FF2BE8D0182FE6D87B08224A013BE3
:10790000DB0002929A589446002ADDD0029AD318DE
:107910005B68002BD8D00878002802D14B78012B67
:1079200002D10624122FCFD107AFAB886978009718
:107930006446AA68A047041EC6D1AB78029A5B08C9
:10794000013BDB00D318390030005B689847041E08
:107950000BD1AB78042BB6D0039A310010782200FB
:10796000009700F06DFB0400AEE76A78002AABD107
:10797000AA7805A93B88087130000A704B80FEF791
:1079800047FBA0E71C43FF1F5CBF00111D4B37B531
:10799000050098420BD000290AD1FFF777FF002895
:1079A00005D11948FFF772FF002800D0058037BDC8
:1079B00001291AD1FFF76AFF041EF8D001235B42A8
:1079C0000380A378FF2BF2D0FE2B07D00023E078B2
:1079D0001422009329001E3300F032FBA01C00F09B
:1079E00053FB01235B426380E1E70229DFD10139C8
:1079F00001F0BEF80028DAD12800FFF747FF041E87
:107A0000DFD1D4E7FEFF0000FFFF0000022210B527
:107A1000074B52421A80074801325A809A80DA8016
:107A200000F07EFA044801F025F8002010BDC046A1
:107A3000A864FF1FB17800118D7900110388F7B594
:107A40000400002B02D102252800FEBD426802215D
:107A5000137825485268FEF7A5FD00282ED0234F45
:107A600001253A88002AEFD0802321885B02012576
:107A70009B1A9942E8DC0C2004F02EF8061E31D047
:107A80003B8822889C4600231800019561469DB2E0
:107A9000491989B2AA421BD8002801D062443A8011
:107AA00000233000082208C0210003F0C5FF104A5F
:107AB0001368002B13D100251660C5E76268022108
:107AC00013780C485268FEF76DFD0028C7D1BAE75D
:107AD00060681D014019418101330198D6E71A0001
:107AE0001B68E6E71325AFE7CABF00111A43FF1F63
:107AF000A464FF1FC8BF0011014B18707047C04637
:107B00001C43FF1F14230A0010B51A40194204D069
:107B10000122102101F048F810BD4B06F9D40120D4
:107B200088434000F8E710B514008B0604D5012205
:107B3000102101F039F810BD08230A001A4019423B
:107B400002D14BB2002B0FDA102101F02DF80028E2
:107B500008D02300F2331B78002BECD0F1342378CB
:107B6000012BE8D10020E6E703208907FAD4E2E7F9
:107B7000F0B51F00184B85B01C680190029103926C
:107B8000002C27D1200005B0F0BDA5683301ED1809
:107B90006B89019A934211D3029A93420ED8002F17
:107BA00004D10A9B002B10D12C00EBE73B00297875
:107BB000039A6868FEF7F6FC0028F2D10136B6B2E7
:107BC000A388B342E1D82468DAE7A3680A9A5B89FC
:107BD0001380E9E70026F3E7A464FF1F37B50C0024
:107BE0000A8849880123914217D3002A15D0651DC0
:107BF00023792A0002210A48FEF7D4FC102300282A
:107C00000BD023796188208800242A000094FFF794
:107C1000AFFF0A23A04200D0230018003EBDC0469B
:107C2000CABF001113B50A00088849880123884299
:107C30000BD8002809D00024137905320094FFF7EF
:107C400097FF0A23A04200D02300180016BD13B5E9
:107C50000A0008884988012388420BD8002809D0E7
:107C60000024137905320094FFF782FF0A23A04213
:107C700000D02300180016BDF0B58BB003904A88E1
:107C800008880E000123824255D3002853D00023D8
:107C9000012704AC23700022718813000092FFF7C3
:107CA00067FF051E3ED02078002835D12B78022BA7
:107CB00018D167706A8983000130E31880005A8008
:107CC00069680222201803F0B7FE23780133DBB283
:107CD0002370042B19D93B006889013080B2002B36
:107CE000D9D01FE002236370122358436A892318F6
:107CF00004305A8069681022201803F09DFE237812
:107D00000133DBB22370002BE5D10C4A6B899B1841
:107D10005A425341DBB2DFE76378012BE4D12B7881
:107D2000022BC7D022780A23002A04D0210003980E
:107D3000FEF798F9002318000BB0F0BD0100FFFF1B
:107D40000F4BF0B504001868002816D083685D89D1
:107D5000A54207D88288AE18B44203DA12019A18F5
:107D6000934201D10068EFE71E005F891036A742F9
:107D700004D1002900D00D801800F0BD3300EFE7DA
:107D8000A464FF1F70B505000C0008880021FFF7F0
:107D9000D7FF03000120002B04D022002800197A0D
:107DA000FFF7C1FE70BDF7B50C0000250190230060
:107DB000EE331B78AB4201D800200AE06B00E65A94
:107DC00000213000E718FFF7BBFF002802D1268012
:107DD0000130FEBD017A0198FFF794FE002802D021
:107DE0003B882380F5E70135EDB2E0E710B50400EC
:107DF00008880021FFF7A4FF03000120002B03D017
:107E00002000197AFFF77EFE10BD0000054B1B68AD
:107E1000002B01D1180004E09A6852898242F6D101
:107E200098887047A464FF1FF0B50E27002687B01E
:107E3000039302ABFF183E8005001F4B40891400DE
:107E4000984207D02B78013000976A6880B2FFF71C
:107E50008FFE060002212B7818486A68FEF7A2FB05
:107E600000280FD06C892000FFF7D0FF002802D037
:107E7000013C0419A4B2039B002B00D01C803000ED
:107E800007B0F0BD02212B780D486A68FEF78AFB27
:107E90000028E7D102212B780A486A68FEF782FBA6
:107EA000002807D0002EDED03B88A342DBD17489A6
:107EB000013CDFE76C89DEE7FFFF0000CABF00116D
:107EC000C8BF0011C6BF001110B50C00FFF7DEFCE3
:107ED00003000220002B0AD0002C00D023609B78E6
:107EE0001720FE2B03D00138FF2B00D1002010BD3E
:107EF00073B50D0001A904001600FFF7E5FF172870
:107F000005D0002E04D129002000FEF727F976BD08
:107F100001221021200000F047FE0028F3D0F6E7F0
:107F2000014B18607047C046B464FF1F37B56B46FD
:107F30009D1D010004000222280003F0B5FD2B88DE
:107F4000B02B0ED12379122B09D12300FA331B78E1
:107F5000012B06D10121608800F0E0F801E01B2B25
:107F6000F8D037BD10B5054B0421187000F098F813
:107F7000FFF74CFDFEF770FB10BDC046B864FF1F55
:107F80000020F0B50BB20F0087B0834234DA274BE4
:107F9000187803F099FE051E2BD00378A02B25D16D
:107FA00003AE3100FEF7E4F8041E0BD1B378DB0713
:107FB00024D51F4B06341B68002B03D03100688882
:107FC00098470400A868002801D003F0B5FC002CF5
:107FD00008D1184A039B1340174A934206D0B3783E
:107FE0001B2B03D00121688800F098F8280003F0CB
:107FF000DBFC80200002784007B0F0BD0F4B1B680F
:10800000002B10D0310068889847041EDAD07378AE
:10801000002BD7D1B27801A90A704B800C71688807
:10802000FDF7F6FFCEE70624F1E7C046B864FF1F70
:10803000B064FF1F00FFFF0000011200B464FF1FC7
:10804000F7B50190FC200D0017001E0003F0A4FC02
:1080500004001320002C12D0B02320002370089BB2
:10806000F4226770658026710830002B08D0190053
:1080700003F0E2FC2100019803F0B6FC0020FEBDF5
:10808000089903F011FCF5E710B5041E06D000783E
:10809000FD2803D803F028FEFF23237010BD000045
:1080A0000A1F93B210B504000220032B05D88240AA
:1080B0000020024BD1529B189C7010BDD864FF1F4A
:1080C0000B8870B5043B04000D000220032B0BD875
:1080D0000121200000F04CFD03001420002B03D0F0
:1080E0002900200000F0DEFB70BD000007B5130082
:1080F000034A00920A00012100F02CFC0EBDC0468C
:108100002983001107B5019203220092024B0A0055
:10811000122100F049FC0EBDA783001107B56B4684
:1081200001AA11800449D88008780633012802D1B9
:10813000190003F0B1FC07BDB964FF1F0C4B10B56B
:1081400018700023FF210B4A1380138193819380C1
:10815000094A53801370517293819372D174D38200
:108160001375517703F088FD00F0FCF910BDC0468F
:10817000E864FF1FD864FF1FBA64FF1FF0B58DB01D
:108180006B46002003910C229B5E834200DBB0E033
:108190005D4B187803F098FD051E00D1A4E003782C
:1081A000902B00D09DE006AF01004688380000F01B
:1081B00013FA79680400002900D19CE03B88052B64
:1081C0006ED13B89032B1CD905AC200000F0A2F82E
:1081D0006288172A61D83989131D994231D179688B
:1081E000237804310291D90738D5607800F08EF9F0
:1081F000071E06D0002303712378012B08D0132B10
:1082000023D0A868002800D178E003F095FB75E042
:108210006288029909A800F0A6F80290380000F0E0
:108220008BF909AA2378387A019200223100009252
:10823000029A00F012F9380000F064F9029B002B5A
:10824000DFD0300000F080F9DBE70378032BD8D1D2
:108250006288029909A800F0D6F8DEE7122B13D144
:10826000029909A800F0B5F8021EEAD127498B88C7
:10827000002BC6D0887909A92378019161780091F3
:10828000310000F0EAF8BCE7002302AA9383300033
:10829000617809AAFFF72AFFB3E71D4B0993F6E7B8
:1082A000042B02D09A1F012AABD8184A043B9B002A
:1082B000995A0029A5D0D218907831003A0000F0E0
:1082C000AEF800289DD13B88042B03D0012130005B
:1082D000FFF724FF012C04D1A868002801D003F087
:1082E0002BFB280003F060FB8020039B000243402F
:1082F00018000DB0F0BD012800D182E70121300047
:10830000FFF70CFFEDE7C046E864FF1FD864FF1FCE
:10831000010017000B7803704B784370CB788A7894
:108320001B021343438070470A88030002700A88C7
:10833000120A42700A88012A06D14A8882704A8845
:10834000120AC2700420704702208242FBD14A8880
:1083500004309A704A88120ADA708A881A718A88F8
:10836000120A5A71EFE710B50400012082420CD9BD
:108370004B780A781B0213432380834206D1CB78C3
:108380008A781B0213436380002010BD022BFBD1AF
:10839000CB788A781B02134363804B790A791B02DE
:1083A0001343A380F0E70B8803700B881B0A43700C
:1083B0004B8883704B881B0AC3708B8803718B8832
:1083C0001B0A4371CB888371CB881B0AC3710820B9
:1083D000704703000120082A14D14A780878120255
:1083E00002431A80CA788878120202435A804A7976
:1083F0000879120202439A80CA79887912020243EC
:108400000020DA80704710B504000120022A05D14F
:1084100000204B780A781B021343238010BDF8B567
:10842000060010200F00150003F0B6FA040001202A
:10843000002C0ED0A0230C22290023806780201D51
:10844000002D07D003F0F8FA2100300003F0CCFA39
:108450000020F8BD03F028FAF6E7F7B51E000090FB
:1084600008AB142017001D78019103F095FA041E43
:1084700012D0A2230370019B47704380099B0571B2
:1084800046710C220830002B07D0190003F0D4FAF3
:108490002100009803F0A8FAF7BD099903F004FA47
:1084A000F6E737B5041E0FD04388002B0CD000250B
:1084B000C1881323007A172201950095FFF7CDFF9D
:1084C000FF2365806372257037BD000010B50C492D
:1084D00004004A88002A09D08B89002B05D000208F
:1084E000CB8A0222834201D010BD012213000A2050
:1084F000434300204032C854C81842800472F3E756
:10850000BA64FF1F0023438003707047094B0021AA
:108510001A0010B55C88002C06D01C79844203D167
:108520000A234B43D01810BD01310A330329F1D17E
:108530000020F8E7BA64FF1F10B50400407A03F08A
:10854000D3FBFF23637210BD7047043010B580B2B7
:1085500003F09AFB002803D00421494203F0F4F809
:1085600010BD000070B50025104CA0682580A581C5
:10857000A580A84202D003F0DFF9A56000250C4CCD
:108580000C4B606D1D80230058331D70A84202D033
:1085900003F0D2F9656500256068002801D003F07A
:1085A000CBF9013508340A2DF6D170BD8065FF1F67
:1085B0002465FF1F7465FF1F70B5041E09D1054DAA
:1085C0002880A881A880A868002802D003F0B4F908
:1085D000AC6070BD8065FF1FF0B54B8885B001931E
:1085E000002343600A7905000F00022A00D07BE0D7
:1085F000CA88032A17D98B685E7819783602DC7826
:10860000D8790E4399781B7A24021B020C4303434A
:1086100053495BBA0B80331D93421ED1042C04D006
:10862000631F022B0ED9012015E0019A4D4B120158
:10863000D35A002B06D00198FFF7BEFF4A4A1369B0
:10864000013313610421B8682E812C80494203F064
:108650007BF86860002005B0F0BD434D042C06D0C7
:10866000631F022B0FD9EB680133EB60DBE7019A44
:108670003C4B1201D35A002B05D00198FFF79CFF09
:108680002B6901332B61374B30000293019B029A17
:108690001B010193002301998C468B521300634404
:1086A0009C8003939E81FFF750FF039B041E9860FC
:1086B00016D00421B868494203F046F8FA88010050
:1086C000043A200003F0B8F90199029AFB888A5A0B
:1086D000043B9B18029A8B522B6801332B60A2E754
:1086E000AB690133AB619EE71E4B0293019B1E01F8
:1086F000029BF35A002B2DD002998C19A0680028F8
:1087000028D0012A26D1FA889B189BB27352A189DE
:10871000994217D39B1AC018B96803F08DF9029BD0
:10872000A289F35A934200D07DE700222B81A388CF
:108730002B80A3686B60029BF2520B4A5368013393
:10874000536070E7084A9368013393600198FFF71C
:1087500033FF68E7044A536901335361F6E7C046C3
:10876000EA64FF1F8065FF1FF064FF1F70B5051EE0
:1087700015D10B4C0B4B1880230058331870606DCB
:10878000002802D003F0D8F86565250050356068F0
:10879000002801D003F0D0F80834AC42F7D170BD06
:1087A0002465FF1F7465FF1FF0B51700A12285B077
:1087B000920001934243394B06001B680C009B1842
:1087C000D933FF331D78FDF741FF0430854204DDC6
:1087D0003000FDF73BFF0430C5B2BD4207D33A007D
:1087E00000213000019B03F0C7FA05B0F0BD29005D
:1087F000380003F099F82300C6B250331E7003937B
:10880000019B29006365380003F03EF9CBB2029367
:10881000002B02D0039B01361E700026230050332C
:1088200003931B78B34204D8606D002831D1002037
:10883000DBE7029A2800002A04D0013B1000B34273
:1088400000D02800F700E719387003F015F97860B8
:1088500000280ED03A78019903F0EEF8019A3B789F
:108860000136D3180E4A0193D369F6B20133D361AE
:10887000D4E7039B18706065A74205D1084A13200E
:10888000D36A0133D362B0E7606803F055F8083467
:10889000F2E703F051F800236365C8E73409FF1FCE
:1088A000F064FF1FF7B50D0007000421686802F0AF
:1088B0004BFF2B89040003702B891B0A43702B8804
:1088C00083702B881B0AC3702E8902250436F6B2EA
:1088D000F42E15D81B4B9F4214D10C2003F05CF8EA
:1088E0001135011E0CD0902303708E3B0371043BA5
:1088F0004380154B8460C680187803F075F8002516
:108900002800FEBD5C237B43104AD31800935833E4
:1089100001931B78002B0FD103003200380000991F
:10892000FFF742FF019B05001B78002BE8D13800C0
:10893000009903F049F9E3E7054A0725536A013333
:108940005362DDE7FEFF0000E864FF1F2465FF1FA0
:10895000F064FF1FF0B587B0009017200F001600DD
:108960000193FFF7F2FD1325041E19D00C98031E86
:1089700002D00199201D9847030AE370052302AA3B
:10898000A0700430908127700098667003A99380CE
:108990000494FFF787FF051E02D0200002F0CCFFF1
:1089A000280007B0F0BD0000F0B587B01F000CAB89
:1089B0001B780391059301210DAB06001C780492EE
:1089C00000F0D6F81425002821D02000FFF77EFD06
:1089D0000135041E1BD01149059B0A780370013232
:1089E000D2B2131EC68001D101231A000B7022716E
:1089F0003000049B03990097FFF7ACFF051E09D1D7
:108A0000230021000648074A093302F0FDFE280032
:108A100007B0F0BD002363802370F8E7EC64FF1F0C
:108A2000A384001130750000F8B505000E00064C57
:108A3000064F2368002B02D03100280098470434E9
:108A4000BC42F6D1F8BDC0469065FF1FA465FF1F6C
:108A50000123064A5B425380002313715362044A88
:108A6000136053609360D36013617047A465FF1F68
:108A70009065FF1F0200002310B506499C000859AD
:108A8000002801D1625010BD0133052BF6D113200F
:108A9000F9E7C0469065FF1F034A5388181A4342FE
:108AA0005841404210407047A465FF1FF0B585B0A3
:108AB00002930AAB1F780CAB1B88009008000E00D5
:108AC00001920393FFF7E8FF05001120002D1BD151
:108AD0000E48FFF7E1FF04001520002C14D00622F9
:108AE0000B99A771E01D02F0A7FF019B30002371D5
:108AF000029B29006371009B66802370039B656263
:108B0000E381FFF791FF280005B0F0BDFFFF0000F3
:108B100010B5FFF7C1FF04000220002C12D06088BE
:108B20000121FFF781FF606A002801D002F0DCFE1E
:108B300028220021200002F0B7FE012300205B4222
:108B40006380207110BD000030B5074A074C55887E
:108B5000010013780020A54204D05B1A59424B4112
:108B60005842104030BDC046A465FF1FFFFF000003
:108B7000084A10B501230C00904208D0FFF78CFF83
:108B8000031E04D0037923405A1E9341DBB2180020
:108B900010BDC046FEFF0000024B1879431E9841ED
:108BA000C0B27047A465FF1F70B504000D00160029
:108BB000FFF772FF002804D10D4B9C4200D0143007
:108BC00070BD416A03790520002907D012221A409E
:108BD000102A02D10520002EF2D10F20DB06EFD59E
:108BE000897E0C20A9428941494249420840E7E771
:108BF000FEFF0000030010B5002800D110BD03489F
:108C0000034A41889142F9D09847F7E7A465FF1FCE
:108C1000FFFF0000002330B5C45CCD5C6C40D45431
:108C20000133102BF8D130BD0F23002210B5C45CE6
:108C300064002243CA54C25CD209013BF7D210BD82
:108C40000200010010B52032103102F065FE10BDA7
:108C5000F0B58BB00390102005931700049102F03B
:108C60003BFF0090102002F037FF009B132401907F
:108C7000002B05D000280CD11324009802F034FEFC
:108C8000019B002B02D0180002F02EFE20000BB03A
:108C9000F0BD102002F020FF0600102002F01CFFA3
:108CA00013240500002E00D1AEE0002819D01022B8
:108CB000002102F0F9FD32002900039802F02CFE99
:108CC000041E0ED133787F2B51D830000099FFF766
:108CD000ABFF009B1B787F2B53D801990098FFF7BF
:108CE000A3FF300002F000FE002D02D0280002F0A9
:108CF000FBFD002CC1D1102002F0EEFE060010207A
:108D000002F0EAFE0290002E7CD0002878D03A00D3
:108D10000F3223000125121105D00F333B4015B24D
:108D20005A4253411BB26A1E1201002B33D0049BDE
:108D3000D2B298180099029AFFF76CFF013D1022F9
:108D40000021300002F0B0FDADB2049F2D017D196D
:108D5000AF4242D0002C33D0300002F0C5FD029B60
:108D6000002B00D189E7180002F0BEFD85E729003D
:108D70003000FFF759FF28002549009AFFF74AFF06
:108D8000A7E729000098FFF74FFF28002049019A24
:108D9000FFF740FFA5E70F210F4004998A18D9B2C9
:108DA0008F4208D9D15C06A819540133102BF6D193
:108DB000029A0199C0E7791A48424141C901F2E794
:108DC0003900300006AAFFF725FF3200039806A9F4
:108DD00002F0A2FD10370400BAE7002CBCD130002D
:108DE000029906AAFFF716FF320006A9039802F0BF
:108DF00093FD082204003100059802F01DFEABE748
:108E00001324A9E71324AAE7002800D06EE733E76C
:108E1000D0BF0011F0B58BB00F00160002250090F6
:108E200000283FD0002A3DD00B1DDBB21800029372
:108E300002F052FE1135041E34D0FDF747FD050047
:108E40003A000099201D02F0E7FDEBB20393E370B6
:108E50002B0CDBB22F0A00936370FFB22B0E237032
:108E6000A7700193FDF72CFD1022010006A802F067
:108E7000D3FD2100029A04AB06A8FFF7E9FE051E08
:108E80000DD1039B08223370009B04A9B370019B92
:108E90007770F370301D02F0BFFDFDF71DFD20005F
:108EA00002F022FD28000BB0F0BDF0B58FB00D0030
:108EB000149E039004920593002A03D102242000FB
:108EC0000FB0F0BD002EF9D00398FFF7E5FD142494
:108ED000071EF4D07278337812021A43B3781B0459
:108EE0001343F27812061A43036A0192934201D3A4
:108EF0000133E3D1002D03D03B7901249B07DED55C
:108F00000822002106A802F0CFFC059B132404339D
:108F1000DBB21800029302F0DFFD051ECFD0059AE8
:108F20000499043002F078FD04223100280002F098
:108F300073FD3900102210310AA802F06DFD2900DE
:108F4000029A06AB0AA8FFF783FE041E0FD108227F
:108F500006A908A802F060FD0822311D08A802F049
:108F60005BFE012807D101990398FDF7C9FC280091
:108F700002F0BAFCA3E70124F9E7000070B51C4C2D
:108F800005002368181E10D0002D14D11A78002A6D
:108F90000CD1981C083202F04FFD02F0BDFD0135E6
:108FA000002808D123681D70012070BD0A33180005
:108FB000082202F041FD2368002BF5D0122002F0B8
:108FC000EBFC061E0DD0C1232168037045700231F1
:108FD0001022023002F030FD23683100587802F090
:108FE00003FD206802F080FC00232360DCE7C0461C
:108FF000CC65FF1FF8B504002020FDF755FB0D4E92
:10900000A700BB590500002B0DD000280BD0D87845
:10901000FF2809D108492A000C55F35907480333A2
:10902000611802F0F1FBF8BD290002F0EDFC002808
:10903000F0D1F8E7E865FF1FD065FF1F4DA20011D2
:1090400070B5064D84006359002B05D0D87802F026
:109050004BFEFF226359DA7070BDC046E865FF1F02
:1090600070B506008CB00C00150000213022684657
:1090700002F01AFC31001022684602F0CDFC1D20DF
:1090800021000322684402F0C7FC6846FFF7D8FDC0
:109090002D21040003222800694402F0BDFC2000B9
:1090A0000CB070BDF0B50700160097B001931CAB73
:1090B0001D7830221EAB00910AA800211C7802F016
:1090C000F3FB102239000AA802F0A6FC10220021AE
:1090D00002A802F0E9FB0722310002A802F09CFC82
:1090E000072202AB9818631E9C41019902F094FC80
:1090F00002AB9C732B005A1E934102AAD37300212A
:10910000102206A802F0D0FB06221D9907A802F043
:1091100083FC1A2002ABC01806221F9902F07CFCC7
:10912000102200990EA802F077FC102202AB0EA9C3
:1091300008781C78013A6040D2B2087001330131DE
:10914000002AF5D10AA8FFF77BFD102212A904001E
:109150000EA802F071FC102206AB0EA908781D784B
:10916000013A6840D2B2087001330131002AF5D1CA
:109170000AA8FFF765FD044310222098E4B212A963
:1091800002F04AFC200017B0F0BD70B50E001400CC
:109190008CB00100102268461D0002F03DFC310039
:1091A000082204A802F038FC2100082206A802F0D8
:1091B00033FC6846FFF744FD04001022280008A98C
:1091C00002F02AFC20000CB070BDF8B506000D00BE
:1091D00000243719AC4200D3F8BD02F095FC030A15
:1091E0003B70631CDBB201379D4203D90234F0545B
:1091F000E4B2EEE71C00EDE773B506000C000225B3
:10920000002819D0002917D0032101A8FFF7DDFF9E
:109210006B469A793F231A40013313436A46300064
:10922000937101A92200FFF71BFF051E04D1032241
:10923000E01C01A902F000FC280076BD0378580765
:10924000DA08C00FD20080009B0710439B0F184321
:10925000C0B2704707230B40C908C9000B43037015
:109260007047000070B50400FFF7EAFE134DA4003C
:109270006359002B21D0186A002801D002F034FB7A
:109280002B59986E002801D002F02EFB2B59D86E76
:10929000002801D002F028FB2B59186F002801D0BC
:1092A00002F022FB2B59586F002801D002F01CFB62
:1092B000285902F019FB00232B5170BDE865FF1FF0
:1092C0000E4B8000C35870B50C00002B0FD09D686A
:1092D000002D0CD02B78201D0B706B784B70A97C67
:1092E000FFF7B8FF2B7E23726B69E36070BD10221D
:1092F0000021200002F0D8FAF8E7C046E865FF1F19
:10930000014B18607047C046E465FF1F074A030021
:109310008000825810B5002A06D0D088984203D128
:10932000012901D1FFF79EFF10BDC046E865FF1F70
:10933000F0B5264E95B087000B93BB5905000991F7
:1093400012200A92002B31D0D888FFF7A5FB040029
:109350001420002C2AD0280010A9FFF7B1FFBB5918
:109360001E781D6A002E23D00895FDF7EFFA07003E
:109370000020FDF7F1FA0790A379E61D069310ADE2
:109380000CA9089800F0E2FA0EA9280000F0D7FA1C
:109390000B9B0A990493069B09980293079B0396DB
:1093A000019300970EAB0CAAFFF77CFE15B0F0BD41
:1093B000FDF7CCFA06903000FDF7CEFAE31DA77951
:1093C000079310AB06000893DAE7C046E865FF1F75
:1093D00030B50C4C85002A59030085B00120002AC5
:1093E0000ED018006946FFF76BFF2B591A78D88802
:1093F000054B002A00D1054B6A46072100F0D9FB36
:1094000005B030BDE865FF1F3F9900114D9900116F
:1094100030B5094C8500295985B0102268462531A0
:1094200002F00AFB2A591121044BD0886A4600F049
:10943000C0FB05B030BDC046E865FF1FE9990011CB
:1094400030B5094C8500295985B010226846353160
:1094500002F0F2FA2A591121044BD0886A4600F032
:10946000A8FB05B030BDC046E865FF1F279A001174
:10947000F7B54D4F86001020F4590D0002F02CFB7B
:10948000F3592062186A132200286CD0033A29008D
:109490009C6802F0D1FAF3591A780192002A58D147
:1094A0001E6A227D317B944651400122019F114268
:1094B00001D167461740217D914339432175377BA0
:1094C0004F40BC4660460027800701D44F08174034
:1094D000012102208F40227D82433A432275377B4F
:1094E0005740BC4660460027400701D497080F400C
:1094F0000420227DBF0082433A432275627D00270B
:1095000094466046727B42400A4201D167460F4052
:109510000121627D8A433A436275777B5740BC469E
:1095200060460027800701D457080F400220627D63
:109530007F00824317436775767B00227E40760763
:1095400001D4BA080A400426617D9200B1430A435F
:1095500062756A78002A08D06278002A05D0052250
:109560000533DA7700221000FEBD0422297911426A
:1095700005D1A17C114202D10533033AF1E7019AEA
:1095800021782C78002A02D10A0021001400182228
:109590000429E8D8042CE6D805206043034A0533A3
:1095A0001218525CDDE7C046E865FF1FE0BF0011FE
:1095B00010B50A001121024B00F0FBFA10BDC046A5
:1095C000839A00110B0030B587B001AD2B806B463C
:1095D00004001100981D082202F02EFA2A000B2127
:1095E0002000024B00F0E5FA07B030BDAB9A001145
:1095F00010B50A001121024B00F0DBFA10BDC04685
:10960000FF9A001113B50B0011006A4613706B46E8
:1096100004000622581C02F00FFA6A4608212000B6
:10962000014B00F0C6FA13BD1F9B001110B50A00D4
:109630001121024B00F0BDFA10BDC0466F9B001116
:109640007FB505000B4BAA00D4580800002C0FD0A2
:10965000666F237FE28821780396266F0296E66E76
:109660000196A46E0094FDF709FC2800FFF7FAFDAF
:109670007FBDC046E865FF1F10B51721FFF7E0FF6B
:1096800010BD000070B50A000D00064B0221040059
:1096900000F08FFA060029782000FFF7D1FF300094
:1096A00070BDC0464F9A001170B586B000236A465F
:1096B0001370836804001D78681E0A2859D801A910
:1096C00002F07AF9060633373B3F43474B4F5300CE
:1096D000180000F042F9062312284BD000281BD1B5
:1096E0006088FFF7D9F90823002813D04279002AAF
:1096F00047D1264B1A78072312070BD5244B1A683B
:109700000723002A06D01668002E03D0290001AADC
:10971000B04703006A4613706B461B786088002BC5
:109720002AD1FFF767FC06B070BD180000F06CF995
:10973000D4E7180000F087F9D0E7180000F093F99B
:10974000CCE7180000F0ADF9C8E7180000F0C3F945
:10975000C4E7180000F0F6F9C0E7180000F0F6F9C9
:10976000BCE7180000F013FAB8E7180000F013FA8D
:10977000B4E707236A46137069466088FFF782FFE3
:10978000D1E70523012AC5D1024BB8E77564FF1F55
:10979000E065FF1FE465FF1FF8B52C4F8600F35905
:1097A00004000D00002B40D0DA8882423DD15A7867
:1097B000062A33D11A78002A2ED0012099681A6A15
:1097C000097D014206D0157B054203D007225A705D
:1097D0000120F8BD0220014204D0157B054201D0D2
:1097E0000922F4E70420014204D0127B024201D096
:1097F0000B22ECE7164B1B68002BE9D05B68002BB3
:10980000E6D020009847BB5900215B78122BDFD1AE
:109810002000FFF715FFDBE70E4BECE7112A04D120
:10982000002900D032252900F2E7002D08D12000C0
:10983000FFF732F9002803D0102302791343037194
:1098400021002800FDF798FAC2E7C046E865FF1F2F
:10985000E065FF1FE465FF1F70B50E4E8500AB5934
:109860000400002B13D01B78002B11D10A4B1B686E
:10987000002B04D05B68002B01D02000984773595F
:109880005B78122B03D100212000FFF7D9FE70BDB9
:10989000024BECE7E865FF1FE465FF1FE065FF1F73
:1098A000094B8000C3581020002B0CD01A6A002AE4
:1098B00009D09B68002B06D0127A1B7E101C9A429E
:1098C00000D9181CC0B27047E865FF1F70B50300CF
:1098D0000D0014000220002A30D000292ED0137071
:1098E0000B78081D53704B789370FFF7A7FCE0705E
:1098F000012002212B7A23716B7B034063716A7B09
:109900000A401343042263716E7B16403343637134
:109910006E7BF608F600334363712B7B0340A37123
:10992000287B014000200B43A371297B0A4013438D
:10993000A3712A7BD208D2001343A37170BD10B566
:109940000A0001000120FFF7C1FF10BD10B50A0099
:1099500001000220FFF7BAFF10BD70B506000C0031
:109960000220002E30D000292ED07378201D0B70DD
:10997000B3784B70F178FFF76DFC012235792572D1
:1099800071794B1008001340934010400343881036
:1099900010408000C9080343C9000B436373B179C9
:1099A0004B100800134093401040034388100240BE
:1099B0009200C9081343C9000B4321202373FCF70D
:1099C00073FE854201D2122070BD2220257AFCF759
:1099D0006BFE8542F7D823781820042BF4D86378DF
:1099E000012BF1D80020EFE7030010B50220002979
:1099F00009D0002B07D00322481C0A7019000D3231
:109A000002F01AF8002010BD03000222080010B571
:109A1000002B06D0002904D00E32591C02F00CF89D
:109A20000022100010BD030010B50220002909D04B
:109A3000002B07D00422481C0A7019000C3201F0D8
:109A4000FBFF002010BD10B5FFF7DEFF10BD0300C7
:109A50000220002906D0002B04D0052200200A7025
:109A60001B784B70704703000220002B08D00029A0
:109A700006D05B7800200B70013B082B00D9183012
:109A80007047030010B50220002909D0002B07D031
:109A90000622481C0A7019000A3201F0CDFF00208E
:109AA00010BD10B5FFF7B0FF10BD02000B00022083
:109AB00010B500290ED0002A0CD00721197011888A
:109AC00059701188090A997011180822D81C01F0E0
:109AD000B3FF002010BD03000A00022010B5002BC8
:109AE0000CD000290AD099785878090201431180D6
:109AF000901CD91C082201F09FFF002010BD03001C
:109B000010B50220002909D0002B07D00822481CDC
:109B10000A701900921801F08FFF002010BD02009A
:109B20000B00022010B500290BD0002A09D0092112
:109B30001970117818185970511C062201F07CFF19
:109B4000002010BD10B5FFF75FFF10BD02000B0035
:109B5000022010B5002A09D0002907D051781970C9
:109B600011180622581C01F067FF002010BD0300E9
:109B700010B50220002909D0002B07D00A22481C6A
:109B80000A701900063201F057FF002010BD10B511
:109B9000FFF73AFF10BD02000B00022010B5002AAB
:109BA00006D0002904D018005178FFF753FB00209D
:109BB00010BDF0B585B017001E006A4606230500EB
:109BC000080091819380FEF7C0FC1324011E0290CF
:109BD0000CD03800B047041E05D1280001A9FEF7BB
:109BE0006FFA041E02D0029801F0A6FE2800FFF7CB
:109BF00001FA200005B0F0BDF0B504008BB0019172
:109C000015000021102202A801F04EFE334EA700DD
:109C1000B85900283CD0C388A34239D10378002B1F
:109C200036D14278062A18D102000100553235316A
:109C30000C3006ABFFF7A9FA002829D12000FFF766
:109C40002FFE020006A902A801F0F6FE200002A9DC
:109C500001F0C2FF01200BB0F0BD816E002917D0CA
:109C60000B8A112A28D19D420ED101981231093A4E
:109C700001F0D2FF012807D1BB5920009D6EFFF7EC
:109C80000FFE29000200DEE732212000FFF7D8FC9A
:109C90002000FEF701FF061E1BD0416A002918D0E4
:109CA0000B8AAB4215D108220198123101F0B4FFA2
:109CB00001280ED1716A0AE09D42E9D1082201987B
:109CC000123101F0A9FF0128E2D1BB59996E8A7EB9
:109CD000B9E7200001F088FFBCE7C046E865FF1F38
:109CE000F0B56B4D87007E5985B0337802900393B1
:109CF000002B00D087E0B368346A0193707806289F
:109D000017D101221B7D134202D0217B114218D1B1
:109D10000222134202D0217B114251D1042213426C
:109D200003D0237B134200D08BE0019B5A7DEB597B
:109D300091E007380428F8D801F03EFE032E426770
:109D40008300B36E002B03D11C2001F0C5FEB0666A
:109D5000EB599C6E002C1CD010220021200001F039
:109D6000A3FD0298FFF79CFD01002000FFF72DFAEC
:109D700001F0CAFE2082200008211230FFF725FAE8
:109D80000298FFF78DFDA076EB592100D888FFF7E8
:109D90000FFC0822EB591CE0B36E002B05D01A0013
:109DA000198AF0881232FFF70DFC0222019B197DFF
:109DB000EB5911423DD0207B10423AD0073208E0E7
:109DC000F488FCF7DBFD01002000FFF711FC0A22FC
:109DD000EB595A70029B9C002A595378073B042B7D
:109DE00011D8D088FEF758FE00284ED0C3895A08F3
:109DF000D2182849029B0298CB542B59411804339E
:109E0000254801F001FD05B0F0BDFCF79FFD030002
:109E10000120834201D100200393EB59DE88FCF737
:109E20009BFD039902003000FFF7ECFB019AEB5910
:109E3000117D042211420CD0217B114209D00B224A
:109E4000C7E7F688FCF73CFD01003000FFF7EEFBAA
:109E50006BE7019A527D01210A4204D0607B0842DF
:109E600001D00C22B5E702210A4204D0607B0842EF
:109E700001D00E22ADE704210A4204D0627B0A42DF
:109E800001D01022A5E71222A3E7FA225200B0E780
:109E9000E865FF1FEC65FF1F57A2001110B5064BC8
:109EA0001A780423100018401A4200D00348FFF724
:109EB00027FA002010BDC0467564FF1F2043FF1F16
:109EC00070B50400FFF7D4FA051E43D12000FFF758
:109ED0007FFA234EA400A0598268937CDB0708D543
:109EE0000321036A1B790B40012B02D1017F0B4335
:109EF0000377431DD97F8B1E022B0DD8022900D07A
:109F00000121C088FCF790FF042133591A7F597052
:109F10000A431A77280070BD01290CD102231022B0
:109F2000437000210C3001F0BFFC30591021353056
:109F3000FFF74BF9EEE70529ECD10223D118437066
:109F400010220C3001F078FD04233259117F0B43AD
:109F50001377EAE708251828DCD1053DDAE7C04683
:109F6000E865FF1FF0B58BB0059143887E4F9E00DA
:109F7000F45915000493002C15D1012902D00020BA
:109F80000BB0F0BD101D57781678FFF757F9EB6846
:109F9000320002932B7A0499019300903B00200039
:109FA000FCF70CFFEBE7E388049A934201D008200A
:109FB000E6E72378012B00D1D4E0059B581E092841
:109FC00000D9CFE001F0F8FC05CE0A29CC506C8511
:109FD0009AB229000498FFF773FFD1E72000290007
:109FE0001022453001F028FDB9594B78042B02D1DD
:109FF000013B4B70C3E70B000A00253335320C31AF
:10A000000498FFF795F90498FFF702FA0522431E1A
:10A010009841BB59C0005A70B2E7200029001022B5
:10A02000553001F009FD049B4F4C9D0029590498BF
:10A030000A0006AB55320C31FFF77AF92959102284
:10A04000453106A801F0E8FD012808D10498FFF782
:10A05000F7F90590002804D106222B595A7005986B
:10A060008EE708230593FAE763780C2B7AD1E36E29
:10A07000002B03D11C2001F02FFDE066BB59D86EE8
:10A0800000286FD01022290001F0D6FCBB5904989B
:10A09000DC6EFFF705FC0D22A076BB595A706EE707
:10A0A000E06E00285ED063780D2B5BD12B880822F0
:10A0B0000382A91C123001F0BFFCBB599A68517D84
:10A0C0000222114226D0186A407B104222D00C3264
:10A0D000E4E763780E2B45D1236F002B03D11620C4
:10A0E00001F0FAFC2067BB59186F002803D010223A
:10A0F000290001F0A1FC0F22BB59CFE763780F2B99
:10A1000030D1206F0622691C103001F095FCBB593C
:10A110009A68517D0422114203D0196A497B114289
:10A12000D5D100210498FFF78BFA28E7636F002B45
:10A130000DD0BB59586F0028F3D01022290001F030
:10A140007BFC0122BB5952425B6F1A61E9E7142084
:10A1500001F0C2FCBB5960675B6F002BE9D126E7B9
:10A160002978DFE707200BE7E865FF1F10B5064CED
:10A17000207001F031FB06212078FDF791FF0348A4
:10A18000FEF778FC10BDC046FB65FF1F0D93001164
:10A1900000200BB270B50D00834216DA264B1878FA
:10A1A00001F092FD041E0DD00378922B0ED0A02B4F
:10A1B00037D0224B1878FF283AD0210001F014FC48
:10A1C000002835D180200002684070BD43780E2BF6
:10A1D0000BD03E2BEDD18378052B12D0082BE8D184
:10A1E00081798088FFF7D8FA08E0154B82889A4277
:10A1F000DFD183681878591CFEF7C0FE002817D1FC
:10A20000D7E7104B1B785B0712D50F4B1B68002B51
:10A210000ED09B68002B0BD0C289811D8088984787
:10A22000ECE7FFF741FAA068002801D001F084FBB9
:10A23000200001F0B9FBC5E7FB65FF1F1943FF1FB5
:10A24000182000007564FF1FE465FF1F10B500783B
:10A25000FFF712FA10BD10B50078FFF7FDFA10BD38
:10A260000C234343084A10B59B185A68002A03D0B0
:10A27000012901D1904710BD9B68002BFBD000291C
:10A28000F9D19847F7E7C0461866FF1F01238340BE
:10A29000094A10B5946B1C439463506B9843506308
:10A2A000D46B20009843012901D120001843D063CA
:10A2B000116B0B43136310BD00800040F0B5002408
:10A2C0000127154B85B0DA6B144E03921A6C01927C
:10A2D000DA64019BE3403B4217D0039DE5403D40DB
:10A2E0000295E5B202992800FFF7BAFF316A736A56
:10A2F000002908D03900002B01D0029979402800AC
:10A30000FFF7C4FF01E0002BF9D101340C36172C04
:10A31000DFD105B0F0BDC04600800040FC65FF1FE6
:10A32000064B01215A68C2400A4204D01B68C34050
:10A330001800084070471B6DF9E7C04600800040D8
:10A340000122064B8240002903D0D9680A43DA6013
:10A350007047D9689143D960FAE7C0460038004099
:10A3600030B5032444430F4BE25C1B199C785D78A5
:10A3700001232D1B0135AB40013BA340A140DB4332
:10A380000C00122807D80849920052181168194089
:10A390002143116030BD054A11680B40234313600F
:10A3A000F8E7C04627C0001108F0004014F0004054
:10A3B000C21F70B5D4B20623092C0BD80125084C56
:10A3C0009540002908D00021FFF7CAFF23682B43DE
:10A3D00023600023180070BD2368AB43F8E7C04634
:10A3E00000380040214BF0B51B185B78022B21D1BF
:10A3F000032444431E4A1F4EA35C12199478012281
:10A4000015008540B76B013CE4B23D43A240B56303
:10A41000194C122815D89B0000290CD117495B183C
:10A4200099680A439A600123205C154A83401168A9
:10A430000B431360F0BD11495B1899689143996013
:10A44000F1E70E4B00290DD159690A435A61225C8C
:10A450001328E8D00123203A93400A4908680343AF
:10A460000B60E7E7596991435961F0E7FC65FF1F0D
:10A4700027C00011008000406CC0001100F00040B7
:10A48000A0F00040A4F00040F8B500241B4E1C4D85
:10A490001C4B1B5D012B1FD1194A9269E2401A42E5
:10A4A0000BD00122B25693402200143AD2B2022AB3
:10A4B00009D815494A6913434B61013402360C35FA
:10A4C000172CE5D1F8BD0022B2560F499200521860
:10A4D00091680B439360F0E7022BEED1E7B23800AE
:10A4E000FFF71EFF01235840C1B23800FFF77AFF83
:10A4F0003800FFF715FF6877DFE7C046F9BF0011A6
:10A50000FC65FF1FFD65FF1F00F0004001220238BF
:10A510008240054B002903D059690A435A617047AC
:10A52000596991435961FAE700380040F8B50E00C7
:10A5300001210F008740114A0400D368FD43BB434B
:10A54000D360831E8B4201D8FFF7E0FF002120007B
:10A55000FFF72EFF0A4A0B4B5168012E05D13943F4
:10A560001B1951605E700020F8BD29405160022225
:10A570001C1962709A6915409D61F4E7003800402B
:10A5800000800040FC65FF1F012210B58240074B90
:10A59000002906D019680A431A600121FFF7C6FF97
:10A5A00010BD196891431960F7E7C046008000406C
:10A5B0000C2370B5002543430A4A29009B181D70DF
:10A5C000094B04001B185D70FFF7B0FF0123A34087
:10A5D000064928000A681A430A6005490A689A432E
:10A5E0000A6070BD1866FF1FFC65FF1F34800040C5
:10A5F0003080004070B504000E00FF2813D0032502
:10A600000540FFF7D5FF084AA3089B009B183F228F
:10A61000ED00AA40AE401968200091433143196013
:10A620000121FFF78DFE70BD18380040F8B50C24ED
:10A630004443134B0500E4186368002B03D1A3685F
:10A640001220002B1AD0022201270E4B00215B1989
:10A650005A7028002770FFF769FF63681E1E08D034
:10A66000A3683E00002B04D02800FFF759FE4640A7
:10A67000F6B228003100FFF709FE0020F8BDC04601
:10A680001866FF1FFC65FF1FF7B5C420FF222B4B88
:10A6900080001958002491433F3A0A431A508022FF
:10A6A000274F5202274E1A60274B1D5D002D21D0E7
:10A6B000A31E012B03D80121E0B2FFF727FF012DD4
:10A6C00018D11F4B9B69E3402B4213D0E3B2180013
:10A6D0000193FFF725FE01000198FFF755FFE3B254
:10A6E000143B022B1DD801217156184A8D40536925
:10A6F000AB4353613B7F002B0DD0E5B22800FFF741
:10A7000095FF2800FFF70CFE7B7F0100834202D0FB
:10A710002800FFF7A5FD01340C370236172CC3D1F2
:10A72000F7BD012100237156F3568D40074A9B0067
:10A730009B189A68AA439A60DCE7C04600E100E0F3
:10A74000FC65FF1FF9BF0011FD65FF1F00F0004011
:10A7500010B501210400FFF7E9FE0123044A00209F
:10A7600011194B70A34091690B43936110BDC04612
:10A77000FC65FF1F70B50E0015000400FFF718FF01
:10A780000C236343094A20009B189D605E60FFF71D
:10A790004DFFF021064B074A8900051E5A5002D092
:10A7A0002000FFF705FF280070BDC0461866FF1F98
:10A7B0000000FF1FBDA2001170B5134D07202C78BB
:10A7C000002C1FD1982221005200280001F034F8FB
:10A7D0000123C420FF222B700C4B80001C635C63A0
:10A7E0000B4B1C605C600B4B195891433F3A0A437A
:10A7F0001A50802252021A600D20074A074901F0C0
:10A800002BF9200070BDC046FC65FF1F0080004092
:10A81000A0F0004000E100E089A6001189A4001129
:10A82000030010B50620072B09D8054A137001F064
:10A83000FBF8D7210020034B034A89005A5010BD72
:10A840004843FF1F0000FF1F8D1BFF1F70B51D0039
:10A8500002240C2910D8094ACA40D2070CD5FBF7AC
:10A860002FFF041E08D1059A04992800FBF744FF26
:10A87000FCF7B2FDFFF712FB200070BD12100000C4
:10A8800030B50D7802232C009C43184201D02B4395
:10A890001C0008252300AB43284201D02B00234392
:10A8A00020241D00A543204201D01C4325002A235B
:10A8B0000D70184204D011781E3B0B43137030BD4D
:10A8C0000028FCD10C2113788B43F7E7F8B51D0065
:10A8D00006AB1B88140007AA0E000B201778002B6C
:10A8E00027D10A78022A49D14A68507811780002A3
:10A8F000244A08438018042840D801F05DF8031268
:10A900001D1B2300F06801F077F8021CC0B2B842AA
:10A9100000D93A1CD2B22000F1682A8001F08CF8EC
:10A9200006E00222F3681B882A8023701B0A6370EA
:10A930000020F8BD0622EEE701232B80F3681B7888
:10A940002370F5E7F368002B16D008222A801A88B6
:10A9500022701A88120A62705A88A2705A88120AE3
:10A96000E2709A8822719A88120A6271DA88A2715A
:10A97000DB881B0AE371DBE72B80D9E701202B8002
:10A98000D7E7C04600D6FFFFF7B516000A781D00CE
:10A9900008AB1F880C000123022A18D14A6850789E
:10A9A000117800022B4A0843801803280FD801F0C1
:10A9B00003F802254439E06801F01EF8C0B207230D
:10A9C000B84204D37B190193152B02DD0D23180027
:10A9D000FEBDE0682A003100C01901F02DF86B4679
:10A9E00000209B88E268D0541B4B1B68834203D035
:10A9F0001B68834200D098470023E8E70B23002F11
:10AA0000E5D1022DE2D1737832781B021343E2685C
:10AA10001380114B1B68002BEED01B68002BEBD072
:10AA20000120E8E70B23002FD1D1062DCED12A003B
:10AA30003100E06801F000F8DEE70B23002FC6D1FB
:10AA4000012DC3D132787533012AC0D8E3681A705A
:10AA5000D2E7C04600D6FFFF0868FF1F70B50C00A4
:10AA60001500072837D800F0A7FF041436361B3628
:10AA7000242E182015290BD8184E1622002130003C
:10AA800000F012FF22002900300000F0D5FF002066
:10AA900070BD18200229FBD11288114B1A80F6E7ED
:10AAA00018200829F4D10A000E48290000F0FCFF04
:10AAB000EDE718200129EBD10B4B10780B49DA692F
:10AAC000FFF7DEFEE3E718200129E1D1064B1078FD
:10AAD0000749DA6BF4E70220DAE7C046F067FF1FA8
:10AAE000C643FF1FBC43FF1F4C43FF1F7443FF1FA0
:10AAF0009443FF1F030010B50020DB0704D5072196
:10AB0000024A034800F08CF810BDC04684C0001112
:10AB10004C43FF1F054A03001068002803D08288B9
:10AB20009A4201D1806870470068F6E7006AFF1F0B
:10AB30000A88030008009A4204D08A8804309A42A6
:10AB400000D0002070470000F8B5F22200230D4F1E
:10AB50000D4E7968050042433370994200D07B6006
:10AB60000A4C0021200000F09FFE00231A007C60A8
:10AB7000AB4202D100203370F8BD01332280DBB23A
:10AB8000F234F5E7F86AFF1FF66AFF1F046AFF1F39
:10AB900073B56B4601900600684615001980FCF7F6
:10ABA0004DFF041E11D1002D0FD07689002E11D03B
:10ABB0000C2000F091FF00280ED0084A04601368B2
:10ABC00086808560002B02D11060200076BD1A00BF
:10ABD0001B68F7E70224F8E71324F6E7006AFF1F73
:10ABE000012100220A4B10B549420A4C1980998074
:10ABF0009A719A70084B2070012019805A60FFF7F3
:10AC0000A3FF2078FCF778FF0448FDF733FF10BD61
:10AC10001068FF1F006BFF1FF86AFF1FCDAC00110B
:10AC2000022310B5002802D0FFF7B2FF030018007E
:10AC300010BD0000030010B50020DB0704D504217F
:10AC4000024A0348FFF7A4FF10BDC04698C0001198
:10AC5000CC43FF1FF0B50E2687B003930CAB1F88C3
:10AC600002ABF6180500080031000292FDF768F803
:10AC700004000120002C0FD03088FFF74BFF0300A9
:10AC80000E20002B08D05E68002E05D02100280081
:10AC9000039B029A0097B04707B0F0BD0A4B10B56E
:10ACA000984207D10122002352420A808B708A8089
:10ACB0008B7110BDFFF73CFF0028FAD001235B42E7
:10ACC000038000238370F4E7FFFF0000F8B5050060
:10ACD00001290AD1134E00243388F227AB4219D040
:10ACE00028001149FFF7DAFF06E0022904D10139F3
:10ACF000FDF73EFF0028EDD0F8BD3B0063437268CE
:10AD0000D018D35A002B09D03A00002100F0CCFD16
:10AD10000134E4B2054B1B78A342EED801235B4219
:10AD20003380DDE7F86AFF1F1068FF1FF66AFF1F18
:10AD300010B5FFF7FDFE03000020834200D0987895
:10AD400010BD0000F0B589B01C000EAB80CB0390A5
:10AD50001E8810AB1B78049202930B7A0D00DB0661
:10AD600016D42B780593022B24D00498FFF7D2FE3B
:10AD7000002812D003689C46002B0ED0029B2200B4
:10AD8000019329003B00644603980096A04705E024
:10AD90000498FFF7BFFE002802D10E2009B0F0BDD5
:10ADA0008368002BF9D00A222900039898470028CD
:10ADB000D7D0F3E76B6858781A786B4B00021043D2
:10ADC0009842D2D8043B984210D2684B984242D065
:10ADD00015D8674BC0180128C7D80B20002EDDD12D
:10ADE000EB681A7859683A80200028E0614BC01857
:10ADF000032800D979E000F0DFFD846A789E5E4B7D
:10AE00009842B2D10B20002EC8D101233B80EB68C1
:10AE100031001B7823706889013080B2FCF790FF05
:10AE20003A88031E0ED0017802328A183A8042898D
:10AE300062704289120AA27059680278E01C00F020
:10AE4000FBFD06E004323A8031000422601C00F071
:10AE50002BFD0020A2E70B20002E9FD1EB6807A955
:10AE60001E8804233B80330A300026706370FCF791
:10AE700067FF051E28D004AB9A890E2304A95B182E
:10AE80003E49C668FCF7D0FF00280BD12B783C4820
:10AE90006A680599FBF786FB002803D1012304AA01
:10AEA0005B42D3813278022A06D17168201D00F0FE
:10AEB000C3FD3B8802333B800E2304AA9B181B88EA
:10AEC000A3701B0AE370C4E704ABDE81F4E70B2038
:10AED000002E00D062E7E9680398FFF729FF0223FC
:10AEE0003B802070000A6070B3E70B20002E00D07A
:10AEF00054E70222EB681B883A8023701B0A6370B8
:10AF0000A7E7E86800F078FDC2B203000720B2426C
:10AF100000D243E70DD00299DBB27118994202DBEF
:10AF2000921BD3B20293029BE9681A003B808919F5
:10AF30005AE70023F6E70B20002E00D02EE7072269
:10AF4000EB683A801A7822705A7862705A88A27038
:10AF50005A88120AE2701A792271DA886271DB88E3
:10AF60001B0AA37175E7C0460429000002280000EF
:10AF700000D8FFFFFFD6FFFF03280000FFFF0000FF
:10AF8000C8BF0011F0B58DB06B460020089120229B
:10AF90009B5E83423DDAA64B187800F095FE071EB3
:10AFA00032D00378B02B2CD10079023816281FD864
:10AFB00000F0EAFB17001E001E001E0031001E00FC
:10AFC00096001E001D011E0052011E0073011E008E
:10AFD000CD011E0050021E001E001E008E021E002B
:10AFE000E302944B94491B8878880B80FBF71AF88E
:10AFF0003800FCF79BFF914B1B68002B01D03800F9
:10B000009847380000F0D0FC8020089B00024340A5
:10B0100018000DB0F0BDEE220021874800F044FC7E
:10B020000BAA3B7B7989388900923A000D32FCF7F4
:10B030009FFD0400804B1B78002C3FD146E0804BE5
:10B04000788805937F4B4100CB5A0BAE073BDBB2B0
:10B0500032880293002301937B4B210006930093D7
:10B06000059BFFF76FFE744D002810D1069B3A8AAE
:10B070001B889A420BD138000599123000F0CCFDA4
:10B08000002804D02B7862899B00EB185A80162385
:10B0900006A81B18328820007989FCF7C5FE2B789A
:10B0A00004009A00AA1851880029C3D00133DBB2EA
:10B0B0002B70002807D006A9C98A9180634A12889C
:10B0C0009A42BCD802E0012149429180002B04D071
:10B0D00059497888FAF7DAFF8AE73E890A2479E045
:10B0E00000253E89574B06937B88069A5B009B5A46
:10B0F000033B9D4202DB002DF0D05BE0162206A848
:10B1000012183B7B798900923A0030000D32FCF72F
:10B110002FFD0590002858D04689017A7888FCF7E1
:10B12000F1FC041E44D1464B78880793069B4100EE
:10B13000C95A454B0439C9B206AAD28A069302916C
:10B14000019400930599079BFFF7FCFD041E2FD186
:10B15000069B39491A88931C002D26D14B8079888B
:10B16000384B4900CB5A5119033B8B4220DD059BDC
:10B1700031485B8941190B71A91C0135C9B2EDB287
:10B18000059145191B0A2B71059B2D49043318188D
:10B1900000F052FC2C4B059A1B88D318DDB22C4BC7
:10B1A0009E4205D00136B6B29CE749889942D6D076
:10B1B000002D0CD0204C2800618800F095FC2070F8
:10B1C00021007888FAF772FF12E7059CF0E7002C5F
:10B1D00000D183E77B78142B00D109E716493B792E
:10B1E0004E800B700C717888FAF712FF00E7162476
:10B1F00006ABE41821003889FCF7A2FD011E00D13E
:10B20000B7E1788822880F4C45002C5B0A4D013C41
:10B21000E4B2029400240F4B01940095FFF792FDD5
:10B22000041E00D014E129007888FAF74FFFDFE60A
:10B23000006BFF1FB842FF1F1868FF1F0C68FF1F3D
:10B240000C69FF1F4864FF1FFC69FF1FB642FF1F08
:10B25000FFFF00001A68FF1F162406ABE418210048
:10B260003889FCF76DFD011E00D182E178882288C3
:10B27000AE4C45002C5BAE4D013CE4B202947C899F
:10B28000AC4B01940095FFF75DFD041E00D0DFE09C
:10B2900029007888FAF724FFAAE60025A44B1D8030
:10B2A0003B00F6331B78A24A78880792AB4208D954
:10B2B0009E4B12880693069943005B5A013B9A42C3
:10B2C00003DB0799FAF716FF92E616246B00FB18CA
:10B2D000059306ABE418059B21001889FCF730FDA7
:10B2E000011E03D1059B01241E8973E77888924BC8
:10B2F0002288069C099343001B5B904E013BDBB206
:10B300000293002300960193099BFFF71BFD041E87
:10B3100002D0059B1E895DE77B88069A5B009B5ADD
:10B32000079A108832881218934202DC1B1A013BDC
:10B3300033807F4C023032880999001900F07CFB81
:10B340002388328801359B182380EDB2A8E70BAA29
:10B350003B7B7989388900923A000D32FCF708FC72
:10B3600000250590059B002B04D10A24002D00D157
:10B370006EE060E0059B7888197AFCF7C3FB01005A
:10B38000041E63D1694C6C4B788806940993069B24
:10B390004400E45A694B063CE4B20BAE3288079392
:10B3A0000294019100930599099BFFF7CBFC041EC1
:10B3B0004CD1079B5E491B881A1D002D30D14A8055
:10B3C000059B5B4C5A8963191A716B1C9BB2E3187D
:10B3D000120A1A71162306A832881B187989059853
:10B3E000FCF722FDFF21AA1C2E1D03350B00059042
:10B3F00092B2B6B2ADB2002803D006ABDB8AD9B2A6
:10B400001B0AA218651911712B714C4D301D2A8829
:10B410004949201800F010FB2B88F618B5B2A1E7B7
:10B420004988914207D17A8806995200525AEB18FE
:10B43000053A9A42C4DC3E4C2800618800F074FA58
:10B44000207021007888FAF75FFED1E5002DF2D157
:10B450003E89BFE6162606ABF61831003889FCF7A0
:10B460006FFC3D000400FA3500282DD0037A9B06BE
:10B470000CD400227B893989788800923A000C32FA
:10B48000FFF7E8FB041E10D03E8915E03088FFF777
:10B4900041FB00281AD08368002B17D0210012220C
:10B4A00078889847041EE4D0EEE72B78002B02D171
:10B4B0007888FAF739FE00262B78002B00D097E524
:10B4C000002C00D194E585E60124DDE70E24DBE7BE
:10B4D000162506ABED1829003889FCF731FC041E4F
:10B4E00047D0037A9B0611D4154A7B88118899426C
:10B4F00003D01448814207D11380134BF2261D78E4
:10B500000023D9B2A94221D30924A1E72888FFF753
:10B5100001FB00282FD08368002B2CD021001222A1
:10B5200078889847041EDFD092E7C0464864FF1F22
:10B530001868FF1F1A68FF1F0C69FF1FFC69FF1FB7
:10B54000F86AFF1FFFFF0000F66AFF1F3100594332
:10B55000546801336018615A0029D2D13C00083484
:10B560002100F22200F068FA21007888FAF7E4FD61
:10B570003EE501246CE70E246AE71D4B1A887B88A0
:10B580009A4231D07888FAF7E1FD31E5F223059847
:10B5900051684343CD18C95A00291FD03B7A012B6B
:10B5A0000BD16C88AB887888AA1D0094FFF752FBFA
:10B5B000041E02D000233B722E88F22200212800B4
:10B5C00000F072F900232B80059B0133DBB2059359
:10B5D000084B05991B78064A8B42D7D801235B425A
:10B5E0001380002CCED0F5E5002634000596EFE759
:10B5F000F86AFF1FF66AFF1F70B504000E00150001
:10B60000FFF796FA031E08D131000548FFF790FABC
:10B6100003001120002B02D01C8000209D7070BD03
:10B62000FFFF0000F8B50B4F06003B780D0014003B
:10B63000FF2B0ED00A2000F0AFF9011E09D0B12374
:10B640000380002346800371C5800481387800F0B0
:10B65000CBF9F8BD0D44FF1FF7B50F0008A9060090
:10B66000088809A90B240988002821D10234022B5B
:10B670001ED1557813782D021D432B008B43019367
:10B680007334002B14D1FB68300019000093FFF7CE
:10B690004FFB019C85420BD02A0030000099FFF738
:10B6A000ABFF041E04D12A0030007989FFF7BAFFEE
:10B6B0002000FEBDF0B50E7885B003900AA805887D
:10B6C0000120022E0DD14C682778647824023C4377
:10B6D000054FBC4205D10398DBB201960095FFF7F8
:10B6E000BBFF05B0F0BDC04602290000034B10B5FA
:10B6F0001B68002B00D09847FEE7C046046BFF1F75
:10B7000007B501A8FFF7F2FF044A05480021121A05
:10B7100000F092F8F8F7B0F8FEE7C046086BFF1F9C
:10B720001044FF1F0000000001B40248844601BC21
:10B73000604700BFF94C010001B40248844601BCD7
:10B74000604700BFEDA5000001B40248844601BC7B
:10B75000604700BF5549010001B40248844601BC5E
:10B76000604700BFADAE000001B40248844601BC92
:10B77000604700BF851F000001B40248844601BC39
:10B78000604700BF3555000001B40248844601BC43
:10B79000604700BF313BFF1F01B40248844601BC33
:10B7A000604700BFF938FF1F01B40248844601BC5E
:10B7B000604700BF75A9000001B40248844601BC7F
:10B7C000604700BF2D2EFF1F01B40248844601BC14
:10B7D000604700BF8D12000001B40248844601BCDE
:10B7E000604700BFC926000001B40248844601BC7E
:10B7F000604700BF2146010001B40248844601BCF5
:10B80000604700BFD532FF1F01B40248844601BC27
:10B81000604700BFA946010001B40248844601BC4C
:10B82000604700BF2124000001B40248844601BCE7
:10B83000604700BFF30E000001B40248844601BC1B
:10B84000604700BFB70E000001B40248844601BC47
:10B85000604700BF8552010001B40248844601BC24
:10B86000604700BFC9A9000001B40248844601BC7A
:10B87000604700BFED4A010001B40248844601BCA4
:10B88000604700BF6D30FF1F01B40248844601BC11
:10B89000604700BF056A000001B40248844601BC4D
:10B8A000604700BF5952010001B40248844601BC00
:10B8B000604700BF154D010001B40248844601BC39
:10B8C000604700BF691F000001B40248844601BC04
:10B8D000604700BF3139FF1F01B40248844601BCF4
:10B8E000604700BF0D52010001B40248844601BC0C
:10B8F000604700BF014C010001B40248844601BC0E
:10B90000604700BFC51D000001B40248844601BC69
:10B91000604700BFDD66010001B40248844601BCF7
:10B92000604700BFE548000001B40248844601BCFE
:10B93000604700BF090E000001B40248844601BC04
:10B94000604700BFD949010001B40248844601BCE8
:10B95000604700BFC56D010001B40248844601BCC8
:10B96000604700BF5D17000001B40248844601BC77
:10B97000604700BF8B52010001B40248844601BCFD
:10B98000604700BF8530FF1F01B40248844601BCF8
:10B99000604700BFF137FF1F01B40248844601BC75
:10B9A000604700BF1D4D010001B40248844601BC40
:10B9B000604700BF434D010001B40248844601BC0A
:10B9C000604700BF1D3BFF1F01B40248844601BC15
:10B9D000604700BFA54F010001B40248844601BC86
:10B9E000604700BF4550000001B40248844601BCD6
:10B9F000604700BF594F010001B40248844601BCB2
:10BA0000604700BFDD52010001B40248844601BC1A
:10BA1000604700BF5147010001B40248844601BCA1
:10BA2000604700BF4551010001B40248844601BC93
:10BA3000604700BF8D1BFF1F01B40248844601BC54
:10BA4000604700BFE94C010001B40248844601BCD4
:10BA5000604700BF6D36FF1F01B40248844601BC39
:10BA6000604700BF0D31FF1F01B40248844601BC8E
:10BA7000604700BF3D37FF1F01B40248844601BC48
:10BA8000604700BF017F000001B40248844601BC4A
:10BA9000604700BF090E000001B40248844601BCA3
:10BAA000604700BFE117000001B40248844601BCB2
:10BAB000604700BF810E000001B40248844601BC0B
:10BAC000604700BFED3AFF1F01B40248844601BC45
:10BAD000604700BF4D1F000001B40248844601BC0E
:10BAE000604700BF3D4B010001B40248844601BCE1
:10BAF000604700BF350E000001B40248844601BC17
:10BB0000604700BFC94A010001B40248844601BC35
:10BB1000604700BF2951010001B40248844601BCBE
:10BB2000604700BFD91B000001B40248844601BC35
:10BB3000604700BF4936FF1F01B40248844601BC7C
:10BB4000604700BF3D36FF1F01B40248844601BC78
:10BB5000604700BF1D3AFF1F01B40248844601BC84
:10BB6000604700BF3D18000001B40248844601BC94
:10BB7000604700BFE538FF1F01B40248844601BC9E
:10BB8000604700BF993AFF1F01B40248844601BCD8
:10BB9000604700BF9DA9000001B40248844601BC73
:10BBA000604700BF1D4B010001B40248844601BC40
:10BBB000604700BFB139FF1F01B40248844601BC91
:10BBC000604700BF6571010001B40248844601BCB2
:10BBD000604700BF3119FF1F01B40248844601BC11
:10BBE000604700BF311B000001B40248844601BC1D
:10BBF000604700BF091B000001B40248844601BC35
:10BC0000604700BF291C000001B40248844601BC03
:10BC1000604700BFAD32FF1F01B40248844601BC3B
:10BC2000604700BFCD4C010001B40248844601BC0E
:10BC3000604700BFC521000001B40248844601BC32
:10BC4000604700BF6DBC000001B40248844601BCDF
:10BC5000604700BF5522000001B40248844601BC81
:10BC6000604700BF055E000001B40248844601BC85
:10BC7000604700BF456B010001B40248844601BC27
:10BC8000604700BF7918000001B40248844601BC37
:10BC9000604700BFE928000001B40248844601BCA7
:10BCA000604700BF2526000001B40248844601BC5D
:10BCB000604700BFC53AFF1F01B40248844601BC7B
:10BCC000604700BF5125000001B40248844601BC12
:10BCD000604700BFF54E010001B40248844601BC34
:10BCE000604700BF156B010001B40248844601BCE7
:10BCF000604700BF1147010001B40248844601BCFF
:10BD0000604700BF093BFF1F01B40248844601BCE5
:10BD1000604700BFB54C010001B40248844601BC35
:10BD2000604700BFB352010001B40248844601BC21
:10BD3000604700BF0124000001B40248844601BCF2
:10BD4000604700BF7139FF1F01B40248844601BC3F
:10BD5000604700BFB14E000001B40248844601BCF8
:10BD6000604700BF0534FF1F01B40248844601BC90
:10BD7000604700BF350E000001B40248844601BC94
:08BD8000604700BF0519FF1F19
:10BD8800000101030202030304030502060207027D
:10BD9800080209030A030B030C020D000E030F032C
:10BDA800100311031303140315001600313C00118E
:10BDB800653C00110000000002000000CABD00112F
:10BDC800192A0F180A000000F1590000FD2400008C
:10BDD800414601007D81001191A10011E575001116
:10BDE800817F00113554001185AF00118150001179
:10BDF800413E0011713F00110000000016160000BE
:10BE08000200000014BE0011F4FFF3FFD2FC000092
:10BE1800B140001100000000000000005475796175
:10BE28000042312E39003030313500676974687549
:10BE3800622E636F6D2F7076767800544830350027
:10BE4800020000005CBE0011292A282A272A262A77
:10BE5800252A242A0A180000E204000071020000C2
:10BE680078EC000005000000744000001027000076
:10BE780060F000000400000006640000204E00008E
:10BE880000000000060000005C44000010270000CD
:10BE98006CEE000007000000050000001F501D00A8
:10BEA800023CB4000001150019000000A1020000C6
:10BEB80030313233343536373839414243444546D8
:10BEC80000000000395800118D58001100000000D2
:10BED80002000000E4BE00116F2A6E2A1A18EAD880
:10BEE800BC80F0FC60000000000000000000F303CC
:10BEF800B59747D6F613F7D777E6F0A7F47400009E
:10BF080001A00000000000006410B71DC8206E3BAF
:10BF1800AC30D9269041DC76F4516B6B5861B24D48
:10BF28003C7105502083B8ED44930FF0E8A3D6D6B2
:10BF38008CB361CBB0C2649BD4D2D38678E20AA01A
:10BF48001CF2BDBDFB349B5F800000800010000028
:10BF580000000000E7610011717800110B62001108
:10BF6800797C00118F6200114F7C0011056300116C
:10BF7800257C001157630011ED7D0011BF6300118E
:10BF8800ED7D0011F1630011A77D0011056300111B
:10BF9800DD7B00117D630011857D0011000000002C
:10BFA8000000000063640011857D0011C564001164
:10BFB80089780011052A042A012A002A022903285F
:10BFC80001280028011800180000000000000000E7
:10BFD80000000000000000870101020102010102C7
:10BFE800010203030401030101010101030302012A
:10BFF80003000D000E0010001100130014010701CA
:10C0080008010A010B011C011D02040205020702B6
:10C01800080219021A021C021D0301030203170079
:10C028000201000504000807000B0A001716001D8E
:10C038001C010201010504010E0D01111001141368
:10C04800011716011A19020201020B0A020E0D024B
:10C058001110021413021716030504030807030B33
:10C068000A030E0D0001020307090A0B0E0F101137
:10C0780012141718191A1B1F20212200CDA800110D
:10C0880089A900110000000002000000CEBF0011C5
:10C0980000000000B5B6001100000000020000001A
:04C0A800CCBF0011F8
:020000041FFFDC
:1000000000000000A93D0011D0BD0011CCBD0011C1
:100010004061FF1F00000000000000000000000021
:1000200000000000000000000000000000000000D0
:1000300000000000000000000000000000000000C0
:1000400000000000000000000000000000000000B0
:1000500000000000000000000000000000000000A0
:100060000000000000000000000000000000000090
:100070000000000000000000000000000000000080
:100080000000000000000000000000000000000070
:100090000000000000000000000000000000000060
:1000A0000000000000000000000000000000000050
:1000B0000000000000000000000000000000000040
:1000C0000000000000000000000000000000000030
:1000D0000000000000000000000000000000000020
:1000E0000000000000000000000000000000000010
:1000F0000000000000000000000000000000000000
:1001000000000000000000000000000000000000EF
:1001100000000000000000000000000000000000DF
:1001200000000000000000000000000000000000CF
:1001300000000000000000000000000000000000BF
:1001400000000000000000000000000000000000AF
:10015000000000000000000000000000000000009F
:10016000000000000000000000000000000000008F
:10017000000000000000000000000000000000007F
:10018000000000000000000000000000000000006F
:10019000F932FF1F5931FF1FC16601000000000046
:1001A000000000000000000000000000000000004F
:1001B000000000000000000000000000000000003F
:1001C000000000000000000000000000000000002F
:1001D000000000000000000000000000000000001F
:1001E000000000000000000000000000000000000F
:1001F00000000000000000000000000000000000FF
:1002000000000000000000000000000000000000EE
:1002100000000000000000000000000000000000DE
:1002200000000000000000000000000000000000CE
:1002300000000000000000000000000000000000BE
:1002400000000000000000000000000000000000AE
:10025000000000000000000000000000000000009E
:10026000000000000000000000000000000000008E
:10027000000000000000000000000000000000007E
:10028000000000000000000000000000000000006E
:10029000000000000000000000000000000000005E
:1002A000000000000000000000000000000000004E
:1002B000000000000000000000000000000000003E
:1002C000000000000000000000000000000000002E
:1002D000000000000000000000000000000000001E
:1002E000000000000000000000000000000000000E
:1002F00000000000000000000000000000000000FE
:1003000000000000000000000000000000000000ED
:1003100000000000000000000000000000000000DD
:1003200000000000000000000000000000000000CD
:1003300000000000000000000000000000000000BD
:1003400000000000000000000000000000000000AD
:10035000000000000000000000000000000000009D
:10036000000000000000000000000000000000008D
:1003700001B70011000000000000000000000000B4
:10038000000000000000000000000000000000006D
:10039000000000000000000000000000000000005D
:1003A0000000000000000000000000000D1BFF1F07
:1003B000000000000000000000000000000000003D
:1003C000000000000000000000000000000000002D
:1003D000000000000000000000000000000000001D
:1003E000000000000000000000000000000000000D
:1003F00000000000000000000000000000000000FD
:08183800106FFF1F4118FF1F94
:10184000024981F3088802F03FFB0000106FFF1F80
:1018500070B500241E491F4A1F484C6308CA1B0567
:101860001B0DE4188242F9D11C4B80228B630021AE
:1018700009201B4B920519621A4B1B4DDA671B4B53
:10188000DA688243DA609A68194802409A60112047
:10189000296002F08DF8112002F06AF880226B6C4A
:1018A000112093436B64EE23DB006343114A1B0C4E
:1018B00013840122104B9A7201F004FC0F4B1B7829
:1018C000002B04D10E4B1021187802F09DFB70BD47
:1018D000000005408805054000060540FF010000A6
:1018E00000F0004004E100E0003800403CF000401F
:1018F000FFDFFFFF1061FF1FC461FF1FF263FF1FC7
:10190000F061FF1F10B502F057FB072804D0122822
:1019100008D0022808D010BD044A0420136B0133FC
:101920001363F8E70220F6E71420F4E7F064FF1FE2
:10193000F8B507000C0026002500503630785135E8
:10194000002804D10300287058342370F8BD29788A
:10195000CA00481E8141A3183800A25C5B68C9B266
:10196000FFF7D0FF00280DD12B78DA00A218013341
:1019700050602B703378044A013B3370136A013393
:101980001362D8E70123DFE7F064FF1F5C234343C2
:10199000074910B5C9180B0058331B78012B05D126
:1019A000FFF7C6FF034A936A0133936210BDC04636
:1019B0002465FF1FF064FF1F10B502F0CDF8064A42
:1019C0000121130010CB4942D967044B136002F088
:1019D000E3F8200010BDC04600E100E01000100058
:1019E00010B5040002F0B8F8024B1C6002F0D4F805
:1019F00010BDC04600E100E0431E5A425341A02200
:101A0000F0B5D2015B421340154D164A40019B18B8
:101A10002A18127E8BB00191002A1BD01A000832BE
:101A2000D46F0022E6B206AFE4B294420EDC28186E
:101A3000C369002B08D0019902AA117106AA049269
:101A400002AA167303A898470BB0F0BD1978B954D1
:101A50000132EAE71A7D1A7806AB01261A70E6E72A
:101A6000B067FF1F00400040F0B5254B0400400167
:101A7000C25C85B0002A2BD01A18117E002927D00D
:101A8000917E002924D01179022921D11689D78885
:101A9000D168F51BADB22A1C102D00D9102292B2CC
:101AA000BE4217D11818012303710023C269C380F5
:101AB00003819A4206D068460321037301710293A1
:101AC00001A890470820002C00D0192001F0FAFA54
:101AD00005B0F0BD013C65426C41A0256442ED01BA
:101AE0002C40084D1B186419074D0633013A92B279
:101AF000AA42EDD01888461C1E80085C2070F5E7CD
:101B0000B067FF1F00400040FFFF00000F220E4B98
:101B100010B59868104002380A280BD801F0FEFF73
:101B20000D0A0B0A0A110A0A0A0A060002210020FD
:101B3000FFF762FF10BD0121F9E70020FFF794FFD6
:101B4000F8E7DB6FF6E7C046004000400F220E4B7F
:101B500010B59868104002380A280BD801F0DEFF53
:101B60000E0A0B0A0A120A0A0A0A060002210120BA
:101B7000FFF742FF10BD01210800F9E70120FFF740
:101B800073FFF7E7DB6FF5E70090004013B5334CC8
:101B90002378072B3DD8324B1A78324B002A39D1A3
:101BA0008022196852020A431A60252001F0C0FE03
:101BB00020232D4A11680B43802113606B460422B9
:101BC000C90508680733104228D080210422C905BE
:101BD000C86810422ED080212020C905CA688243DF
:101BE000CA6014221A701A78002A2FD18021C905E0
:101BF000C86820320243CA6014221A701A78002A78
:101C000028D11A4B1A7D22785A601D221A70593237
:101C1000DA6013BD1A6816490A40C5E7086802432E
:101C20000A6014221A701A78002ACED01A78013A63
:101C3000D2B2F7E7C8680243CA6014221A70197852
:101C40004A1ED2B21A700029F9D1C4E71A78013AB3
:101C5000D2B2C7E71A78013AD2B2CEE74843FF1FA3
:101C60001044FF1F3CF000404043FF1F0020004095
:101C7000FFFFFEFF564B70B51B68012B03D1554A81
:101C8000936D0133936502F03FF9534B534A18604B
:101C9000534B544C1A600123534A1360534A136048
:101CA0002378002B06D006225149524802F014F93D
:101CB00000232370504A514B10681B78C1B2002B8F
:101CC0000ED14F4CC0B223785BB2002B4FDB237890
:101CD00024785BB264B21B0424021B191B18136026
:101CE0000B1C50294ED95023464A47491078DBB285
:101CF000FF2202284BD10868444C454D267890437A
:101D00002A78964254D9227824782E78023B5D10A6
:101D1000A31B6B435201D31A10335B1118430860A5
:101D200001F012FF031F012B45D83A4B1B78002B03
:101D300006D0394B1B78002B02D0002002F0B4F8FB
:101D4000A122364B92009978354B4A431B689B1869
:101D5000832292009B181B78033B012B03D8AF20F2
:101D6000400002F011F801222E4BDA8270BD237878
:101D700024785BB264B2FF33FF341B0424021B19C6
:101D80000138ABE7CAB2022AAED20223ACE7086838
:101D9000254C264D267890432A78964208D92278F9
:101DA00024782D78023B5B10641B63435201B2E739
:101DB0002378DBB2B2E70228D5D11D4B1B78013B5B
:101DC000022B03D91B4B1B78022BCCD16C20C8E70C
:101DD0009809FF1FFC0FFF1F3C64FF1FFF3F00001F
:101DE000141003404064FF1F0C1003400010034018
:101DF000D50BFF1F7211FF1FB40003408C09FF1F9A
:101E0000680AFF1F490AFF1F94000340460AFF1F8C
:101E1000470AFF1FF908FF1F2209FF1F300DFF1F90
:101E20003409FF1FBC0BFF1F440AFF1F450AFF1F99
:101E30001C09FF1F2309FF1F10B501F0FDFF002241
:101E4000014B1A8010BDC0463864FF1F10B502F068
:101E500023F8A121054A89009478054A6143126854
:101E6000044B5218528C1A8010BDC046300DFF1F13
:101E70003409FF1F3864FF1F10B50D4B0D4A9978C8
:101E8000A1239B004B431268D218531DD97F0A4BE4
:101E90001B88994209D2441C07D0C82805D0D269B2
:101EA0005B1A5A43054B5343C01801F025FF10BD80
:101EB000300DFF1F3409FF1F3864FF1F710200003F
:101EC00070B5244D2B68002B28D002F035F82B6814
:101ED000D8402B680400002B27D001F0BDFF2B68F1
:101EE000D8401D4B1D4A9978A1239B004B43126893
:101EF000D118D25C91239B00002A20D0CA5801320D
:101F0000CA50174B17491B680868834214D3D23B49
:101F1000181A012A1AD0144B186070BD02F00CF880
:101F2000124B196801F090FED3E701F095FF0F4BBB
:101F3000196801F089FED4E70D495B18E8E7CA503B
:101F40000C4B1B68DB68E418201AE4E7F530FF301F
:101F5000E1E7C0461C08FF1F300DFF1F3409FF1FBB
:101F60009C09FF1F3C64FF1FA009FF1F1808FF1FEB
:101F70002DFF3F004464FF1F70B504000D002829A9
:101F800016D10300A433C2881B889B1A0B4A9BB24C
:101F900093420DD906006A3605223100653001F002
:101FA0001BFF002804D13100200001F085FF70BD27
:101FB0002900200001F088FEF9E7C046FE7F0000FE
:101FC000F8B50500012001F04FFE134CA36AA26A88
:101FD0009342FBD1114E336002F006F81049030022
:101FE00008601048426894460F4A17680022BC45B2
:101FF00001D24268BA1A0D4802603268AD18A422B4
:10200000E562606A520302436262094A1278002A5A
:1020100001D00F3B0B60F8BD00F00040340AFF1FF9
:10202000E408FF1F28100040180AFF1F1C0AFF1FAA
:102030001C09FF1F70B580241025E405A3682B43FD
:10204000A36001F081FEA368AB43A36070BD0000F4
:10205000F7B5160080221C001023D205019191686B
:1020600005000B43936000225A4BD7301A6001F0F1
:1020700083FE9D232A002F009B00EB58CA320121CA
:102080000092FC37002B01D00021009A386801F043
:102090009BFF2900009BCB311A784F4BD3351A6038
:1020A0004B780A781B0213438A7812041A43CB78C0
:1020B0001B061343494A1BBA13604B790A791B026A
:1020C00013438A7912041A43CB7931001B06134358
:1020D000434A1BBA13606B782A781B021343AA7811
:1020E00012041A43EB781B0613433E4A1BBA1360D3
:1020F000019A330213433C4A13603C4B22001B1BE2
:102100009C4603293DDCB3089A0013005142B21AE1
:10211000032A46D1354AE018511A827840781204D1
:1021200000020243E05C043302430A600022FF2BFA
:102130004BDDF0222E4B12011A600F222D4B1A603C
:102140002D4A1368002BFCD00023224A2749136034
:10215000091B321D0B191B68043A180A23706070A2
:10216000180C1B0EA070E3700434002AF2DC8022ED
:1021700010213B68D20501333B6093688B43936029
:10218000F7BD6346D578981893782D061B042B432A
:10219000157804392B43557804322D022B43036004
:1021A000AFE7022A0AD1114AE05C511AE2185278CC
:1021B000120202430A6004339BB2B7E7012AB5D189
:1021C0000A4A521AE15C1160F5E7084959180A6099
:1021D0000433ACE7000004403C00044038000440F5
:1021E00034000440300004400C000440000104406E
:1021F000040004401000044014000440F7B515002A
:1022000080221C001023D2050091916807000B4327
:1022100093600023654AD730136001F0ADFD9D2324
:102220003E009B00F9583B00CA363200FC330029BF
:1022300000D07FE0586801F0C7FE390032785C4B6F
:10224000CB311A604B780A781B0213438A78AC466C
:1022500012041A43CB78281D1B061343554A1BBA98
:1022600013604B790A791B0213438A7912041A43CB
:10227000CB791B061343504A1BBA13604B7A0A7A78
:102280001B0213438A7A12041A43CB7A21001B06DD
:1022900013434A4A1BBA1360009A2B021343484A5D
:1022A00013602200474B1B1B0093009BCE785B18EA
:1022B00001938B7836061B0433430E78043833437E
:1022C0004E78043136023343019E33600328ECDC40
:1022D0000321A808431C9B002940800003292BD11F
:1022E0003849E5185E18A9786D78E35C09042D0279
:1022F000294319433160030008330021FF2B2DDDF2
:10230000314B324919600F21314B196001232749A4
:102310000B60304B19680029FCD006211B680B406C
:10232000042B20D080220020D20593680A318B43F1
:102330009360FEBD01217DE7022908D121495D1886
:10234000E1184978E35C090219432960D3E70129C0
:10235000D3D11C495918E35C0B60CCE71948181815
:1023600001600433CAE7002310490B606346002B69
:102370000CDC3B00FC335A68102101325A60802289
:10238000D205936801208B439360D2E7009B9B1892
:102390001B68190A13705170190C1B0ED37004239B
:1023A0005B4291709C440432E0E7C0460000044068
:1023B0003C00044038000440340004403000044035
:1023C0000C0004400001044004000440080F000019
:1023D000100004401400044070B5061E19D00222FB
:1023E0005A4B9B799343012B13D1594B1A78FF2AEF
:1023F0000FD15A78FF2A0CD19A78FF2A09D1DA78BE
:10240000FF2A06D11A79FF2A03D15B79FF2B00D16D
:1024100099E0504B0C201A78012A08D000224E4D2A
:102420001A7029780B00093B042B01D8212070BDBC
:102430004B1F012BFAD9454CA37B042B00D982E01A
:10244000A279032A00D97EE09A1ED2B2012A02D8CC
:1024500060881F2877D9002E56D0012E73D1A0880E
:102460000128E3D0002907D1581E032803D801F022
:1024700055FB121715122E702978481E032811D803
:102480000025364B1D602823237501F02DFCA84242
:1024900027D0A580CAE702212970EDE70421FBE7D8
:1024A0000321F9E707390129C0D82D490968C96A0C
:1024B0008906BBD52B4908780028B7D1012A01D954
:1024C000002BB3D102230B708021274D26338901C5
:1024D0002878237501F068FD80212878890101F0B2
:1024E00093FD0123A380214B1B78002B0AD0FA22F5
:1024F00080211F4B92001B8809025A431A4B1878FF
:1025000001F0CAFB002092E701F026FB2B78A680A1
:10251000073B012B03D917482E7001F025FC114B06
:10252000114C1A78002A06D08021002220788901D7
:102530001A7001F039FD01F02FFB8021207809028B
:1025400001F032FDDEE7122071E7C046A60BFF1F47
:102550006B09FF1F1A09FF1F1C09FF1F4809FF1FF6
:102560004464FF1F2309FF1F1B09FF1F2109FF1FD1
:102570002C09FF1F0010004010B5002901D001F008
:102580002BFD10BDF7B5604B01919978A1239B00FD
:102590004B435E4A060014681022E418D6235B0001
:1025A000E0583623FF33E35C00279343222B41D1CD
:1025B000574B0F3A1A600760012501F065FB019B3C
:1025C0001880E8235B00E35C002B01D0B34258DDA8
:1025D0000023504FFB70AD33FF33E3581A68002AD5
:1025E00003D09B88DB439B071DD03823FF33E35C7C
:1025F000002B18D09B235B00E35C002B13D1D1335D
:10260000FF33E35CB3420EDAA4235B00E15AE01827
:10261000090A023101F010FB23000122FE33013EC2
:1026200001351A87FA70E8235B00E35C002B2AD09F
:10263000A8B2FEBD03683D00002BBED081880430E7
:10264000090A023101F0F8FAD6235B00E3581F6053
:10265000B2E72300B133BA00FF33985801378188BD
:102660000430090A023101F0E7FAE8235B00E35C79
:10267000BB42EEDCE822F61AED1800235200A35408
:10268000A6E70027F1E7200001F0AEFB00281FD0ED
:10269000002E1DDD7319882647190193B60020000E
:1026A00001F00AFB5A30800020184068013581880B
:1026B0000430090A023101F0BFFA200001F0ACFC3D
:1026C000A3590133A351BD4202D0019B9D42E6D1E3
:1026D000114BE35C002BABD095239B00E35C002BFC
:1026E000A6D00E4BE15A0029A2D00D4AA35C994214
:1026F00002D90133A3549BE700231A212000A354DD
:1027000001F012FB94E7C046300DFF1F3409FF1F94
:1027100000140340E010FF1F5A0200007202000084
:102720005E0200000D4970B54A6E0D4CD2038B69F4
:10273000D20BA24206D80B4D0224AA4204D901F0C2
:10274000EBFA70BD02246442E21815007E24254095
:102750002242F4D0A3432B438B61F0E700F000400A
:102760000A200000FC1C0000F8B51D4B1D4F1A7814
:10277000002A10D1BA7B002A02D101321A7003E07C
:10278000032AFAD0022AF8D001F0AEFA0022012082
:10279000154B1A70F8BD154B154D1C68154B9E78DE
:1027A00001232B702878C0B200F09EFBBB7B002B6E
:1027B0000BD101F061FAA1239B007343E41883233A
:1027C0009B00E41823782B70E4E7032B02D101F07F
:1027D0005BFBF0E70020022BDCD101F025FBEAE7F0
:1027E0001C09FF1FA60BFF1F2309FF1F3409FF1F32
:1027F000490AFF1F300DFF1FF0B587B00EAD2F78CF
:102800000FAD2D780593AC46634614000E4D0CAA0F
:1028100012782E7803930D9B009201932200059B62
:10282000029701F0B9FA2E70012C01D0042C08D1C6
:10283000802206498B889343054A1278D2011343BC
:102840008B8007B0F0BDC0461C09FF1F6C11FF1F35
:102850007809FF1F0B001B3B70B504003020E02BF4
:102860000DD81300E025493BFF3B9BB2ED00AB4286
:1028700005D8034B200019825A8201F055FB70BD28
:102880008410FF1F10B501F03FFB054B00205B6873
:10289000052B04D9034A5268D20200D4980810BD0F
:1028A00000100040FCE100E070B501F055F90D4B5F
:1028B0001B68FC33DC691D6AFFF7E4FF641984427E
:1028C00004D2094B01241B68002B07D004220024EA
:1028D000064B1A70064A93690133936101F05CF963
:1028E000200070BD4464FF1F9809FF1F2309FF1FCC
:1028F000FC0FFF1F70B50C4D2B68FC335C6A01F0B8
:102900002BF9FFF7BFFF2B680025FC339B6AE31808
:10291000834204D2054B1B68AB4200D1051B01F07A
:102920003BF9280070BDC0464464FF1F9809FF1F93
:10293000D722044B92009B5810B5002B00D098472B
:1029400010BDC0460000FF1F10B501F0CFF8FFF723
:10295000EFFF2749274BCA6D274C1A4084235B00A1
:102960001343CB65254B1B68186A01F07DF9244B96
:10297000244A1A60244B254A1A60A022244B520094
:102980001A60244B187801F0B7FA2000224901F0B0
:102990004BF90023A3600233A360204B204923603E
:1029A00003232048A36001F03FF910221E4BFF20B3
:1029B0001A60802252031A60802292031A608022D9
:1029C00012041A6001F070FA012001F015FBFA20E0
:1029D000400001F0C9FA582001F0D6F9134801F07F
:1029E0007BF9012001F030FA072001F00DF910BD4C
:1029F00000F0004000FEFEFF141000404464FF1F82
:102A0000000003400180063DBC0003403408000084
:102A1000A40003404A0AFF1F71020000C30900001E
:102A2000FFFF3F002810004000E100E0307500008B
:102A3000674E336888331B6883F3088801F09CFA7B
:102A4000644A6549136800200B401360634B644A75
:102A50001B68934200D1A6E001F0D6F90221614A39
:102A600013688B431360FFF76FFF5F4B5F4C187861
:102A7000C0B201F089FA0023A3600233A3605C4B6B
:102A80000120236001F0F0F80323A36001F05CFA59
:102A9000040001F039FA050001F056FA554B1860B0
:102AA00001F0E2F9544B1968621A531EA14200D298
:102AB00013008022D203934201D39B029B0A326807
:102AC000D16AC90700D471E04C491C0C09689BB25B
:102AD0004C4359432402090A641803264849FC322E
:102AE00093680A6847489B1A474A0768126847492B
:102AF0009B18474A9A1833409208DB190A60036012
:102B0000042B03D9013233400A6003600E68414947
:102B1000A619300001F098F83F4F3E493B68C318B2
:102B20003B603000019301F067F93C4E30680818B3
:102B300038493060884205D9019B01333B6001F080
:102B40005BF9316001F040F9354B1B78002B0DD05B
:102B500001F0DAF9334B621B196812188A4232D23B
:102B60004919091B091A304801F05EF82F4E337AD3
:102B7000002B0ED001F0C8F9621BF16812189142C7
:102B800024D94919091B091A294801F04DF80023D5
:102B90003372284B83F3088801F00EF8002001F00F
:102BA00033F901F0D9F901F02FF95CE7DC01990064
:102BB0000234641A5900641A09214B438033CB4014
:102BC000A408E41889E7FA218900CCE71A49DBE771
:102BD0004464FF1F1CF00040FFFFC1FF0C0AFF1FF1
:102BE000B641210310000040490AFF1F14100040A5
:102BF000C3090000100AFF1F340AFF1F380AFF1F15
:102C0000200AFF1F280AFF1F1C0AFF1F240AFF1F9C
:102C1000C4090000710200006008FF1F2C0AFF1F9A
:102C20001C09FF1FE408FF1F00100040740BFF1F6A
:102C30003C10004000000020DC050000A022054BF5
:102C400092009B5810B5002B01D0984710BD01F0A1
:102C5000EBF9FBE70000FF1FA122054B92009B58F8
:102C600010B5002B01D0984710BD01F0DDF9FBE74E
:102C70000000FF1FA222054B92009B5810B5002BAD
:102C800001D0984710BD01F0CFF9FBE70000FF1F0E
:102C9000A322054B92009B5810B5002B01D09847FA
:102CA00010BD01F0C1F9FBE70000FF1FA422054B96
:102CB00092009B5810B5002B01D0984710BD01F031
:102CC000B3F9FBE70000FF1F70B501F01DF94F4B92
:102CD000186000F0E9FF0400C30702D400F04CFFC5
:102CE00070BD00224A4B1A604A4B187801380428FC
:102CF00029D800F013FF0320181C2400200001F045
:102D0000BBF80128ECD0444C2378042B6ED101F0A1
:102D100023F80028E4D001F00FF8582001F034F82F
:102D200002232370DCE7200001F03EF8E9E72000F1
:102D300001F0DAF8E5E7200000F05EFFE1E72000AF
:102D400000F042FFDDE700F0FFFE0500012808D19A
:102D5000324B1B78053B012B03D82000FFF76EFF99
:102D6000D1E72D4B1B78022B01D0052B20D1022D52
:102D700028D12B4B9B7BAB431CD12000FFF76CFF72
:102D8000264B18780128BED16405BCD424492522DD
:102D90004B7B034205D1233A13405A425341263319
:102DA0001A000B7D9342AED9322001F0B5F8AAE7A4
:102DB000022D07D1194B1B78052B11D12000FFF7ED
:102DC00059FFDDE7012D0BD1012B03D12000FFF7C7
:102DD0005FFF98E7062B03D12000FFF767FF92E71C
:102DE000200001F021F9022D8DD1C9E7032B04D178
:102DF0000C4B987C00F0C8FE72E7072B00D06FE701
:102E0000094B987B00F0B0FE6AE7C0469C09FF1FA3
:102E10009809FF1F9009FF1F2309FF1F1C09FF1FAF
:102E2000A60BFF1FBC0BFF1FD40BFF1FFA210A4B81
:102E30000A4A49001A640A4A5A500A4A04395A503E
:102E4000094A08319A64094A5A50094A5C315A5071
:102E5000084ADA667047C0460000FF1FF927FF1FC7
:102E6000F528FF1FA928FF1FD923FF1F6927FF1F70
:102E7000791EFF1F4D1EFF1FF7B50B0CFF27012208
:102E8000009300233C001E001D009446019089B26F
:102E900062469A401000084018413618B6B2FF2F1B
:102EA00002D1012E00D19FB2009802401A41AD1804
:102EB000ADB2FF2C02D1012D00D19CB20133102BF9
:102EC000E6D10320012E07D1012D04D1019B24015D
:102ED000E4191C700138FEBD102EFCD10238102DF3
:102EE000F9D00230F7E700008023F7B59C46264B67
:102EF000264F01932649274A274D284C284B022864
:102F00001AD1604638600868264E30408026360365
:102F10003043086001990978002909D11660224AD6
:102F20002A60224A2260E02219689143A03A1BE0FD
:102F30008021C9021160F2E766463E600F68194EB3
:102F40003E408027FF023E430E6001990978002928
:102F50000DD1176001280ED1154A2A60154A22604A
:102F6000E02219689143C03A0A431A60F7BD8021F4
:102F700089021160EEE7E0210F4A02432A600F4AFE
:102F800022601A688A43F0E74B0AFF1FE000034003
:102F9000D80003409000034000000340500003406D
:102FA00040000340FFFFE3FF0280063D804508220A
:102FB0000180063D80660822008006988055082220
:102FC000F8B51E4B80261A680020140034403242A7
:102FD00032D11A681A4F32431A6001223B68063018
:102FE00093433B6000F040FE0122164D2B681E43C8
:102FF0002E603B680A2613433B608027BF00124BBC
:103000001B683B4211D1013EF6B2FF2E09D17E2250
:103010000E4B1C682B68E40B1440934323432B6036
:1030200005E0082000F020FEE9E7002EEFD1802225
:103030002B68600893432B60F8BDC046C4F0004085
:103040005CF0004018F0004068F0004060F0004084
:1030500010B500F0E1FD01215820034A00F0A4FD65
:10306000FFF7AEFF10BDC046600AFF1F10B5782203
:103070000021034800F0A0FE00F046FE002010BD35
:103080003867FF1F70B5040000F066FD00230C20B8
:103090000B4A010059438D18515C00290DD0A14203
:1030A00008D1012300246B7000F0C6FF00F074FD0E
:1030B000200070BD01330A2BEBD11224F6E7C04685
:1030C0003867FF1F70B5040000F046FD00231900AB
:1030D0001D000D4A1078002806D0A0420CD1557072
:1030E00001310C320A29F5D1002B0AD100F00CFE77
:1030F00000F052FD002070BD5078461EB0411B18F4
:10310000EEE700F099FFF3E73867FF1FF7B504001B
:103110000C20002384460E4D019267465F43E85D14
:103120007E19A04212D000280BD10A4B9C46624661
:103130001B7808331370019B70707C557160B3600D
:10314000FEBD01330A2BE8D10320F9E70720F7E79A
:103150003867FF1F3467FF1F8020F8B5484BC00554
:103160001B68C1248360474BFF251A680123134362
:103170004361454BA4001A68444B40211A60444BFC
:103180001A68444B1A60444B1A59AA431A51C52273
:1031900092009E58AE433143802699509F583F4934
:1031A000F6010F403E439E509E5880273602360A55
:1031B0003043985080201A5900020A4002431A51A5
:1031C00004341A59364E3F04324080263A431A518D
:1031D0001A5936061202120A32431A5108341A5981
:1031E00080260A4002431A51C32292009F58B446D7
:1031F000AF4337439F509F58294E0F4007439F507E
:103200009F58374080263604374380269F509F586A
:1032100036063F023F0A37439F50C0221F59AF4333
:103220003A431A511A591202120A1643C6221E5163
:1032300092009C58AC4365462C439C509C580025FA
:103240000C4020439850C72080001A58154C11405C
:10325000C02212020A431A50134B1B78DB08AB4200
:1032600001DC0020F8BD2378002B06D0A368002BDA
:1032700000D0984701350C34EEE71220F2E7C04643
:103280004443FF1F4043FF1FB0F000403067FF1F63
:10329000B4F000402C67FF1F00E100E0FF00FFFFDB
:1032A000FFFF00FF3867FF1F3467FF1F030010B5E3
:1032B0001F2809D8072200201340072404490A7850
:1032C000A24313430B7010BD00230620F5E7C04650
:1032D0003467FF1F054B06491B780A6805485B07E2
:1032E00002401B0B134300200B6070473467FF1F25
:1032F0001CF00040FFFFC1FF70B50C25FFF7EAFF8F
:103300000A4B1C780A4BE4086543ED18002C01D1E8
:10331000200070BD2B78002B06D06B68002B00D0EE
:103320009847013C0C3DF1E71220F2E73467FF1F9C
:103330002C67FF1F1FB5002102220B000191009195
:10334000052000F051FC02230B490A681A42FCD107
:1033500020230393039B5A1E0392002BFAD1074AA2
:103360001368002BFCDA0B246C442000012100F0D0
:1033700013FE207804B010BD90C8004000C8004083
:1033800013B504000A4B0193019B002B01D11120BE
:1033900016BDFFF7CFFF23000340044205D00520F0
:1033A00000F062FC019B013BEDE71800F0E7C0462E
:1033B000FFFFFF0707B500F0CFFB80220821D205F1
:1033C000936A0191002B01D10739916202210C4AC5
:1033D00011600199481E01900029FAD10331116052
:1033E000053101910199481E01900029FAD111601F
:1033F000002B02D18022D205936200F0CDFB07BDE5
:1034000000C00040F0B52D4C89B02378002B4FD17F
:10341000FEF7D2FA02232A4F03903A681A42FCD1EF
:1034200020230693069B5A1E0692002BFAD1254EA6
:103430003368002BFCDA0120FFF7A2FF011E02D047
:10344000112009B0F0BD030003220190009005ADEA
:103450009F2000F0C9FB0321280000F09DFD0223FE
:103460003A681A42FCD120230793079B5A1E079201
:10347000002BFAD13368002BFCDA0120FFF780FF24
:103480000028DDD10398FEF7ABFAAA786B78110417
:103490001B020B4329780B4363601300113B0A495D
:1034A000052B07D801239340A3600B6001232370F1
:1034B0000020C6E780231B03F6E7C0462C43FF1F0E
:1034C00090C8004000C800409808FF1F1E4B30B550
:1034D0005A6818781D4B85B0D31859424B410121C9
:1034E0000093002300F078FB194B1A4A02259A63D7
:1034F00000221A6510325A658022C4219D65164B40
:103500001648D202DA6789004258154B80241A40C7
:1035100080231B0413434350642341200393E40599
:1035200000F006FA402000F003FA6562039D6B1E6E
:103530000393002DFAD103236362FFF73BFFA562DB
:10354000FFF760FF05B030BD3843FF1F95FFFEF762
:1035500000C80040050001FF04E100E000E100E0D8
:10356000FFFF00FFF0B585B00700FEF725FA022344
:1035700005002D4C22681A42FCD120230093009BA9
:103580005A1E0092002BFAD1284E3368002BFCDA29
:103590000120FFF7F5FE002803D01124200005B01C
:1035A000F0BD234B2360022322681A42FCD1202362
:1035B0000193019B5A1E0192002BFAD13368002B14
:1035C000FCDA0120FFF7DCFE0028E6D1194B1F6072
:1035D000022322681A42FCD120230293029B5A1E26
:1035E0000292002BFAD13368002BFCDA0120FFF79E
:1035F000C7FE0028D1D1104B2360022322681A4253
:10360000FCD120230393039B5A1E0392002BFAD173
:103610003368002BFCDA0120FFF7B2FE041EBCD198
:103620002800FEF7DDF9B9E790C8004000C8004067
:1036300001000006A8C800400180000110B500206C
:10364000FFF790FF10BD000010B5064B18705960D1
:10365000FFF73CFF00211320034AFFF757FD00202E
:1036600010BDC0463843FF1FCD34FF1FF0B5040026
:1036700085B003920291FEF79FF9882263035B0BEA
:1036800052051A438023DB059D6A8023274F009251
:10369000BA68002601901B039A420CD9F823260031
:1036A0001B041E401C4206D08022214B52025E6247
:1036B00019680A431A60002D0BD100F04DFA02225E
:1036C0001C4B1A608023DB055A62013A9A6200F0B3
:1036D00063FA0023039A934220D1002D0AD100F00F
:1036E0003BFA144B03221D608023DB055A629D6266
:1036F00000F052FA8023BA681B039A4208D9002EC0
:1037000006D000220A4B0C495A621A680A401A6015
:103710000198FEF765F9002005B0F0BD009A029906
:10372000D2181278CA540133D4E7C0462C43FF1F85
:1037300000C8004000C00040FFFFFEFFF0B587B0AA
:10374000029103920400FEF737F9019000F004FAA9
:10375000802302250122234EDB0535605D629A62DB
:1037600000F01AFA204F3B682B42FCD1202304932F
:10377000049B5A1E0492002BFAD11C4D2B68002B7F
:10378000FCDA0120FFF7FCFD002802D0112007B071
:10379000F0BD2000039A029900F03EFB02230400D2
:1037A0003A681A42FCD120230593059B5A1E0592C4
:1037B000002BFAD12B68002BFCDA0120FFF7E0FD8B
:1037C000051EE3D100F0C8F980230322DB05356034
:1037D0005A629D6200F0E0F90198FEF701F9E0B24B
:1037E000D5E7C04600C0004090C8004000C8004077
:1037F000F0B5802489B00600FEF7DEF8E405A36A80
:1038000002250393029000F0A7F90123304F3D6099
:103810006562A36200F0C0F92E4C23682B42FCD1F4
:1038200020230593059B5A1E0592002BFAD12A4DA1
:103830002B68002BFCDA0120FFF7A2FD002803D043
:103840001124200009B0F0BD244B2360022322681C
:103850001A42FCD120230693069B5A1E0692002B87
:10386000FAD12B68002BFCDA0120FFF789FD021E3C
:10387000E6D11B4B03211E60030001900090202025
:1038800000F0B2F9022322681A42FCD120230793E8
:10389000079B5A1E0792002BFAD12B68002BFCDAEB
:1038A0000320FFF76DFD041ECAD100F055F98023F7
:1038B0000322DB053C605A629C6200F06DF9039BB9
:1038C000002B01D1FFF776FD0298FEF789F8B8E7E3
:1038D00000C0004090C8004000C800400100000641
:1038E00094C8004007B5000201910422000A01A912
:1038F000FFF724FF0EBD000073B5050005240B4A39
:10390000A3005B429B1819686B46DE1D3000FFF771
:10391000B3FA022804D133782B55013CEFD276BD9F
:10392000052CFCD00128FAD10230F8E71409001167
:103930001F2807D8012380228340D20591680B43BA
:10394000936070473F2808D80123802220388340A5
:10395000D20551690B435361F3E75F28F1D8012386
:10396000802240388340D205116A0B431362E8E796
:103970001F2807D8012280218240C9058B68934304
:103980008B6070473F2808D8012280212038824070
:10399000C9054B6993434B61F3E75F28F1D80122D6
:1039A000802140388240C9050B6A93430B62E8E7E7
:1039B0001F2810D880230200DB05153A1968012A58
:1039C00006D820229143196019680A431A6070478B
:1039D00001228240F6E73F2811D880230200DB0550
:1039E000353AD968032A06D810229143D960D9689C
:1039F0000A43DA60EBE7012220388240F5E75F28CE
:103A0000E5D842238022181A413B8340D205516AEF
:103A100099435162516A0B435362D8E710B50400D1
:103A2000012813D1A022184992050B685B015B099C
:103A300013430B60154B164A19681140154A0A4387
:103A40001A60402219680A431A6010BD0028FCD190
:103A500001000A2000F000F921000B2000F0FCF822
:103A6000C0220A4B920019680A4340211A601A6862
:103A70008A431A60B022044912060B685B015B0995
:103A800013430B60E1E7C04614F000401CF0004017
:103A90007F00FEFF80FD010072B6074A1368013304
:103AA00013600422054B1A600023054A136080222C
:103AB000D2055360FEE7C0467808FF1FC0F0004003
:103AC000C4F0004005490B68002B05D1044A0A6088
:103AD00004490A60044A13607047C046140AFF1F75
:103AE000841E0000380AFF1FC4F000400023034A70
:103AF0001360034A1360034A1360704754F0004098
:103B000040F1004044F1004002B4714649084900C8
:103B1000095649008E4402BC7047C04602B4714643
:103B200049084900095C49008E4402BC7047C04600
:103B300003B47146490840004900095A49008E44BF
:103B400003BC70470000000001B40248844601BC79
:103B5000604700BFDD0C010001B40248844601BC8F
:103B6000604700BF75A9000001B40248844601BC4B
:103B7000604700BFC1F7000001B40248844601BCA1
:103B8000604700BFDD0A010001B40248844601BC61
:103B9000604700BF4DF9000001B40248844601BCF3
:103BA000604700BF9DA9000001B40248844601BCE3
:103BB000604700BF0167010001B40248844601BCB0
:103BC000604700BF7997000001B40248844601BCF9
:103BD000604700BFF935010001B40248844601BCCA
:103BE000604700BFC56D010001B40248844601BCB6
:103BF000604700BF496D010001B40248844601BC22
:103C0000604700BFF535010001B40248844601BC9D
:103C1000604700BFF90D010001B40248844601BCB1
:103C2000604700BFED68010001B40248844601BC52
:103C3000604700BF2D6C010001B40248844601BCFE
:103C4000604700BFC115010001B40248844601BCB1
:103C5000604700BF090E000001B40248844601BC61
:103C6000604700BF61A3001101B40248844601BC53
:103C7000604700BF0189000001B40248844601BCCE
:103C8000604700BFE9F6000001B40248844601BC69
:103C9000604700BFCD0C010001B40248844601BC5E
:103CA000604700BF8B52010001B40248844601BC4A
:103CB000604700BFBD0B010001B40248844601BC4F
:103CC000604700BFD9B0000001B40248844601BC7F
:103CD000604700BF51B8000001B40248844601BCEF
:103CE000604700BF8D11010001B40248844601BC49
:103CF000604700BFA9D8000001B40248844601BC57
:103D0000604700BF8937010001B40248844601BC06
:103D1000604700BFADAE000001B40248844601BC5C
:103D2000604700BFD1AE000001B40248844601BC28
:103D3000604700BF53B9000001B40248844601BC8B
:103D4000604700BF6DF6000001B40248844601BC24
:103D5000604700BFDD3F000001B40248844601BC5B
:103D6000604700BF01D7000001B40248844601BC8F
:103D7000604700BFC1A5000001B40248844601BCF1
:103D8000604700BF8944000001B40248844601BC7A
:103D9000604700BF7912010001B40248844601BCAB
:103DA000604700BF9D6A000001B40248844601BC20
:103DB000604700BF0934010001B40248844601BCD9
:103DC000604700BFB70E000001B40248844601BC42
:103DD000604700BFD544010001B40248844601BCDD
:103DE000604700BFCD4C010001B40248844601BCCD
:103DF000604700BF71B0000001B40248844601BCB6
:103E0000604700BF090E000001B40248844601BCAF
:103E1000604700BF016C010001B40248844601BC48
:103E2000604700BF9573010001B40248844601BC9D
:103E3000604700BF19FA000001B40248844601BC83
:103E4000604700BF8D82000001B40248844601BC77
:103E5000604700BFE512010001B40248844601BC7E
:103E6000604700BF6D0B010001B40248844601BCED
:103E7000604700BFC166010001B40248844601BC2E
:103E8000604700BF0134010001B40248844601BC10
:103E9000604700BF75F8000001B40248844601BCC9
:103EA000604700BFF9ED000001B40248844601BC40
:103EB000604700BFED6B010001B40248844601BCBD
:103EC000604700BF85C1000001B40248844601BCC0
:103ED000604700BF09B7001101B40248844601BC25
:103EE000604700BFE94C010001B40248844601BCB0
:103EF000604700BF0534010001B40248844601BC9C
:103F0000604700BFEDA5000001B40248844601BC33
:103F1000604700BFC95C010001B40248844601BC8F
:103F2000604700BF6137010001B40248844601BC0C
:103F3000604700BF116E000001B40248844601BC16
:103F4000604700BFE90B010001B40248844601BC90
:103F5000604700BF156B010001B40248844601BCF4
:103F6000604700BF8552010001B40248844601BC8D
:103F7000604700BF8512010001B40248844601BCBD
:103F8000604700BFC9A9000001B40248844601BCD3
:103F9000604700BF8914010001B40248844601BC97
:103FA000604700BF3D71010001B40248844601BC76
:103FB000604700BFB352010001B40248844601BC0F
:103FC000604700BFE927000001B40248844601BCF5
:103FD000604700BF2144000001B40248844601BC90
:103FE000604700BFE9D4000001B40248844601BC28
:103FF000604700BFBD5C010001B40248844601BCBB
:10400000604700BF6911010001B40248844601BC49
:10401000604700BF0D52010001B40248844601BC54
:10402000604700BF5976010001B40248844601BCD4
:10403000604700BFE917010001B40248844601BC93
:08404000604700BF21A9000048
:1040480002000000CABF001101000000C0BD00113D
:1040580002000000C6BF0011010000008840FF1FD9
:1040680002000000C8BD001101000000C061FF1F70
:1040780002000000C4BF0011030000003461FF1FEC
:104088001200000002000000CABF00110100000079
:1040980008BE001102000000C6BF001101000000A8
:1040A80005BE00110200000012BE0011030000004E
:1040B8006F61FF1F02000000C4BF00110300000071
:1040C8008461FF1F02000000C6BF0011010000004C
:1040D80004BE00110200000010BE00110300000021
:1040E8004561FF1F02000000C4BF0011030000006B
:1040F8006661FF1F02000000CABF00110100000036
:1041080048BE001102000000C6BF001101000000F7
:10411800D141FF1F020000005ABE0011010000003B
:1041280043BE001102000000C6BF001101000000DC
:10413800D041FF1F0200000058BE0011010000001E
:104148008C61FF1F02000000C6BF001101000000C3
:10415800CF41FF1F0200000056BE00110100000001
:1041680033BE001102000000C6BF001101000000AC
:10417800CE41FF1F0200000054BE001101000000E4
:104188002EBE001102000000C6BF00110100000091
:10419800CD41FF1F0200000052BE001101000000C7
:1041A80029BE001102000000C6BF00110100000076
:1041B800CC41FF1F0200000050BE001101000000AA
:1041C80024BE0011020202020202000000000000E8
:1041D800161500009D4C0011634C0011B8BE00116B
:1041E80090011D0018001800FFFF070102030405D5
:1041F80006020106000000000000000000000000A8
:1042080000000000000000000000000000000000A6
:104218000300000002000000CABF001101000000F6
:10422800D8BE001102000000C6BF00110100000046
:104238008C42FF1F02000000E2BE001101000000D6
:10424800BA61FF1F02000000C4BF00110300000094
:104258002464FF1F02000000C6BF00110100000017
:104268008C42FF1F02000000E0BE001101000000A8
:10427800BC61FF1F02000000C4BF00110300000062
:104288001C64FF1F12A6A6A6000000000000000084
:10429800161500000001000000000111FFFF0000DA
:1042A8005048593600000000000000000B000500CF
:1042B800F0000000B4000028002800283075A00095
:1042C800A000A000A00000080008E001F000100015
:1042D8001000100010001000100050005000500096
:1042E80010001000D0070000000000000F000100BF
:1042F8000500307507001000010081FF0000000074
:10430800FF0000004975001151730011E1700011A0
:10431800FFFF0100FF000000659F0011E19C0011F4
:10432800F99B0011000000000000000000000800D8
:10433800040000003B0001085902E0018821280020
:10434800FF00000002000000CABF001101000000C9
:1043580090C0001102000000C6BF0011010000005B
:10436800C943FF1F02000000C2BF00110100000086
:10437800F067FF1F02000000C6BF00110100000027
:10438800C843FF1F02000000C0BF00110100000069
:10439800C643FF1F02000000C6BF00110100000055
:1043A800C443FF1F02000000BEBF0011010000004F
:1043B800BC43FF1F180018001D00900102000003F5
:1043C8000202000002000000CABF00110100000044
:1043D800A4C0001102000000C6BF001101000000C7
:1043E8000C44FF1F02000000BCBF001100000000C9
:1043F8000000000002000000C4BF0011030000001C
:064408001068FF1F20FFF9
:040000051FFF184180
:00000001FF
